:020000041100E9
:103000007FB50023284C294D03932800217C284AB2
:1030100001F0E1FA002812D103232800217C03AA41
:1030200001F080FA00280AD1224B039A9A4206D175
:10303000214B2248E360224B636104B070BD02263D
:10304000217CFE2228001F4B009601F03DFA00284B
:1030500001D00020F1E71C4BA2899A42F9D1217CD2
:10306000FF222800194B009601F02EFA0028F0D11B
:10307000E389174A934203D1164B17486361DCE793
:10308000164A9342E5D1164B164A1B68934206D95D
:10309000C02304222800217C9B0001F07EFA124B01
:1030A00012486361C9E7C046FC61FF1F3442FF1F3D
:1030B000813700005959530059598320F0BE00113F
:1030C000094200110862FF1F595900000A62FF1FE0
:1030D00083050000BD410011D0BE00118215000023
:1030E0002062FF1F87130000C5420011E0BE0011DF
:1030F000002370B51A4E1B4C30006361637401F0FD
:1031000091F9402323744B2B0CD9CC233821AC22CA
:1031100030009B01217401F040FA00280AD00025FC
:1031200025740CE0FFF76CFF051E08D1237C0433E7
:10313000DBB2E7E70C4B0D4D63610D4BE381236878
:10314000002B08D1002D06D00C222900200008F009
:10315000ABFC2B7B6374300001F0A2F970BDC0465C
:103160003442FF1FFC61FF1F5D420011C0BE001111
:10317000AAAAFFFFF7B5164B0192C318021D002043
:10318000009388235B05D3181B685C1C1AD09CB283
:10319000402C18D88D781E0CAC466746CD782D0291
:1031A0003D43AE4206D1019800280ED110000C70AC
:1031B000240A4C7003249BB20733A343D218009B0C
:1031C0009A42DED3FEBD4432F9E71000FAE7C0466A
:1031D000FC0F0000802213B503000324019189B283
:1031E000520107319B18A14304305A1A88235B050A
:1031F000C3181B68591C03D190429241104016BD60
:1032000099B2402907D80B000733A343C018904256
:10321000ECD30020F3E74430F9E7134B134A1B6863
:10322000126810B5FA24934201D81A00F824104B02
:10323000E4021B689A4210D813000E4A12689A42A0
:103240000ED3013307D1F823DB029C4203D10A4994
:10325000054808F089FC200010BDFC24E402ECE7DE
:10326000FE24E402F7E7C04600C0071100D00711B2
:1032700000E0071100F00711FFFFFF7FF0B59BB0E2
:10328000150004900391402A00D9A0E006AB5980B4
:103290001A80FFF7C2FF0400042816D9002206A9ED
:1032A000FFF768FF052810D906AB1B88AB420CD18D
:1032B000002D07D0514B2A000499C01808F074FA69
:1032C000002802D101201BB0F0BD06AB1D802000FC
:1032D0000699FFF77FFF041E7BD1069B0793FFF73C
:1032E0009CFF80235B01C618802307001B039E42BE
:1032F00001D3F826F60288235B05F31801931B68B7
:10330000013302D0019808F067FC3D49019808F0AC
:103310002BFC3B1D0293331D05938822029B520513
:103320009B181B6808935A1C3CD044219AB2009108
:10333000402A04D80320D11D814389B2009103990A
:103340001B0C8B4224D0402A22D80122300008A92D
:10335000FFF710FF021E1BD1380008A9FFF70AFF74
:103360000400042831D9009A059B9B188022520141
:10337000B218934240D288235B05C118009A09A86D
:1033800008F092FB1D4B009A09A9F01808F0BCFA4E
:10339000009A029B9446634402931A4B029AFB18CC
:1033A0009A42BAD388235B05FC1821680198013939
:1033B00008F0DAFB200008F00FFC039A07AB5A80F4
:1033C00030000799FFF706FF0400002C03D100200E
:1033D00079E70428FBD988235B05E018069908F0F3
:1033E000C3FB0323EA1C9A4300D16BE7034B049908
:1033F000E01808F089FA65E70424ECE704000011FE
:10340000FFFFFF7FF80F0000F7B505001400402A0A
:1034100021D8002701AE71803780FFF7FEFE042817
:1034200016D93A003100FFF7A5FE042810D93688D6
:10343000BC420BD0BD4209D0221CB44200D9321C80
:10344000064B92B2C118280008F02EFB30B2FEBD28
:10345000C04300B2FBE703204042F8E7040000113C
:1034600037B5042204000D0001A81649FFF7CCFF70
:10347000020004280BD1019BA34208D3AB4204D025
:10348000104901A80195FFF7F9FE01203EBD0E4C41
:1034900023682000019308F09FFB01992000013967
:1034A000019108F061FB80235B01E418074B9C420B
:1034B000EED10422034901A80195FFF7DFFE0020A9
:1034C000E4E7C0465555000000C007110000081190
:1034D00030B589B008F0F8FB10226946254808F09D
:1034E00023FC254B009A9A420ED1019B029A0F2B86
:1034F00033D8002101240698013B08D2002900D0CE
:103500000292029B013331D10023029325E0551C26
:10351000F2D102002100EFE710341022200004A9AC
:1035200008F002FC029B013301D1069B0293882321
:1035300004995B05C918059B06981A03120B0491A0
:103540000592814203D02B4201D108F0ADFA019BD4
:10355000013B0193019B002BDED1029B002B03D08A
:10356000049304984168084709B030BDE025014C38
:103570002D03EFE700000111504859368022F8B5BD
:10358000964C974BD200002120001C6008F04CFBA9
:103590002300944A88331A60934B1A786A23002ACE
:1035A00000D01133E3620A232365904B37221B7846
:1035B0000820A3638E4B2118E361102323628D4BF7
:1035C0003B256361C823DB00A36123008C331A60B1
:1035D0002823013AE26320646364CA67043A211D28
:1035E000CA672100BC310D602100C0310860210094
:1035F000C4310B6021000635CC310D602100083D3F
:10360000C8310D602100D0310A602200D432106030
:103610002200D832136022000227E0322100176016
:103620004222DC310A6021001B3DE4310D602100A3
:10363000E83108602100EC310B6023000521F433F0
:1036400019602300F0331A602300183290331A6097
:1036500023009433186023001E3A98331A60AF2376
:10366000DB002360644BFA262363644B644DE36004
:10367000644BF031A3642300FF31FC33B600A1603A
:1036800021611E60A5627325E5656D3D6565A565D3
:1036900096255D4AAD00E264666258606766A5667D
:1036A00000270925A767E566584F594D6067200038
:1036B0002567E2673A6015279C30676007001A208B
:1036C00038602000A0300700212038602000A8309A
:1036D00007004C4838602000F83006602600642758
:1036E000A436376026005F3FAC3637602600033FC4
:1036F000B03637602600C637B4363760260000275C
:10370000B836376038269E60424E96205E64424E40
:103710005A66DE61414E9A645E62F53EFF3E9E62ED
:103720001E269A67354A8000DE661F675F67DD6583
:103730001D661862DA67BE23394A5B00E250394BD6
:10374000D838235004302250C4225200A350C6233C
:10375000E4205B00E1500433334AE1503349344BF9
:10376000D1603449800019503349E938FF38195085
:1037700032490430195032493248D161324911631B
:10378000324951631900F4310860CE2030494000BD
:1037900011603049195019002F48F83108602F493D
:1037A000D16582212E4A89005A501A002D490832CB
:1037B000D1671A002C49B432116088212B4A890044
:1037C0005A501A002A49883211602A4ADA6408F0ED
:1037D000DBF8012008F0B8F9F8BDC0460004FF1F6F
:1037E000AC64FF1F706FFF1F6C44FF1F4A0AFF1F6E
:1037F0003A07000080C3C9019A020000DC050000FE
:103800006A18000050C3000088130000F009FF1F71
:10381000204E00006509FF1F68100000C409000069
:1038200040420F0010270000FC00FF1FB11CFF1FCB
:103830000000FF1F052DFF1F8D30FF1F252FFF1FCD
:103840007120FF1F6127FF1F8D20FF1F3922FF1FDF
:10385000FD1FFF1F8529FF1F6D2AFF1F8D19FF1FE9
:103860009128FF1FB525FF1FC125FF1FFD1EFF1F4C
:10387000B51FFF1F751EFF1F0223F0B50124624D07
:10388000624E2B70624B91B01C70624F0393336891
:1038900000210820BB7006F073FE082006F06AFDC8
:1038A0000023984205D0BA78552A02D0332A00D096
:1038B0009DE03360042006F0DDFF08F095F9FFF786
:1038C0005DFE08F081FA1F2201240021524B10AE48
:1038D0001A70524B1C70524B1970524B196891431D
:1038E000163A0A431A60602219689143403A0A4323
:1038F0001A6008F0F1F807F05FFF4B4B9847C120C2
:10390000FF214A4B80001A588A431A50C522920060
:1039100098588843BF390143995098584449084002
:103920008021C9010143802099509958C00509029E
:10393000090A0143995080213E48490107F094FF4C
:10394000032322003C49019400933C4808F054F8BA
:103950002C223B4905A808F0A7F805AC617820782F
:10396000023406F027FDA642F8D1364C0020012192
:1039700006F034FE2268344B03201A40A023DB02F9
:1039800013432360802322689B041343236022682F
:103990002E4B1A4080239B03134323602C4A2D4B4C
:1039A000934200D8012008F01FF808F04DF9802359
:1039B0002268DB0413432360287807F0B5FF039BDC
:1039C0001878C0B208F040F807F0F6FF224904204A
:1039D00007F05AFF06F01AFF00F040F800F030FE42
:1039E00000F0D8FE00F018FA002011B0F0BD0093EE
:1039F0002100194A042007F09FFF8023DB059C6209
:103A0000FFF766FD56E7C0464A0AFF1F34F0004044
:103A10006C44FF1F2C62FF1F480AFF1F490AFF1F4B
:103A2000680AFF1FBCF00040E1A2000000E100E0D6
:103A3000FF00FFFF7044FF1FF456FF1F7054FF1F6D
:103A4000E8BD001114F00040FF7FF8FFFFFF9FFF6B
:103A50000080FF1F706FFF1F3B000108002210B5A0
:103A60001100112008F050F910BD0000F8B5002336
:103A70000926374F374C3B62E3681120B343E360BC
:103A800007F0D2FF112008F0C7F8112008F014F851
:103A90004023226880251343236080236268DB0271
:103AA00013436360A3682C4A2B43A360A3680221DD
:103AB0001340A3608023A2689B0113431022A360DC
:103AC000236C072093432364236C0F3A134323642E
:103AD00080235B003B62226B204B1A402263626BA7
:103AE0001A406263A26B1A40A263E26B1340E36365
:103AF000E3681B4A1340E36006F05CFC01210720E9
:103B000006F06CFD174B11205A6C15435D6407F0ED
:103B100093FEFD21144B154A89005A508023C7207B
:103B2000626B5B0313436363E36880003343E360CA
:103B30000F4B104A19581140802212020A431A50A2
:103B4000802292051A6008220B4B5A63F8BDC046CA
:103B500000F000403CF00040FFFFDFFFEFFFEFFF11
:103B6000FFFF7FFF003800400000FF1F5118FF1FBC
:103B700000E100E0FF00FFFF00000540E12010B57C
:103B8000C00407F0C9FE10BD70B52B4C238C002B70
:103B90002AD0FA22D200934201D2FFF7EFFF228A05
:103BA000238C002A21D1DA0023826382A382E3825C
:103BB00023836383A383E38322606260A260E26065
:103BC0001E4D1F4A6420EB8093420AD8FA2200203F
:103BD000D200934205D91B4A0A21981807F084FFA6
:103BE000C0B200232872238470BD0720E11CCA7F65
:103BF00001320240CA7705D10325201DC17F013162
:103C00002940C17708325200A352002321001A0034
:103C1000088A01321B180231082AF9D1221DD27FED
:103C20009200A350626823689B18A2689B18E26800
:103C30009B185B099BB2C3E76C61FF1F1462FF1FF7
:103C4000B70B000030F8FFFF30B503A804880B2045
:103C5000002C0ED14968074D0878497809020143C4
:103C60000A20A94205D1012120001980024B1B7AAC
:103C7000137030BD192A00001462FF1FF7B515003C
:103C800008AA16884A680F4F147852781202224305
:103C90000A24BA4214D10122DBB2019200962A0012
:103CA00007F004FD041E0BD1074B1B68002B07D047
:103CB00068782A7800021043424250410130984708
:103CC0002000FEBD022900009861FF1F30B50125CC
:103CD00003790400BFB02B4211D00A49408807F095
:103CE00051F828420BD0084B01A95B8D4D800B8009
:103CF000064B00221B7A60880B7104F023F93FB059
:103D000030BDC0469061FF1FA840FF1F1462FF1F17
:103D100010B50549054806F0EBFF0421044A0548A3
:103D200006F0A8FF10BDC0469061FF1FFFFF000016
:103D300014BE0011A840FF1F10B5024804F084FF14
:103D400010BDC046CD3C0011012303700B4B1A7A05
:103D50004270022282709A78C270DA78027103226D
:103D600042711A7982715A79C2710C2202729A795F
:103D70004272DB7983720B207047C0461462FF1FCA
:103D8000022310B50370013B437005338370103379
:103D90000371443B43712A3383714433C37100235D
:103DA0000372064B04001B8843720A30FFF7CCFFF6
:103DB000831D0A30C0B2E37010BDC0461462FF1FFD
:103DC00010B5142007F0E0FE124B142200211860F9
:103DD00007F02AFF002007F0A7FE012007F09CFE55
:103DE000022007F069FD032004F0D2F9042006F058
:103DF000E7F9052003F010FC062004F0DDF80720A9
:103E000001F0BEFA082006F015FF092001F08AF83B
:103E100010BDC0469C61FF1F07F03EFE012007F069
:103E200093FF07F0D9FF0000094B10B5040098423A
:103E300005D0012904D12000064906F059FF10BD24
:103E40000229FCD1013904F0BDFE0028F3D0F6E7C9
:103E5000FEFF0000C261FF1F70B50D7A100004AABA
:103E60002C00168810221440154220D1002E20D19B
:103E70000A78022A18D14A68517815780E4A090240
:103E80002943914205D00D4A914209D01C800A2451
:103E900004E014220A491A8007F006FE200070BDD3
:103EA0000C2208491A80F7E71C800124F6E7082451
:103EB000F4E70B24F2E7C046F3FF0000F4FF000034
:103EC000F842FF1F0CBF001110B504000749084855
:103ED00006F00EFF074804F0F7FD0020E40704D5C4
:103EE0000721054A054806F0C5FE10BDC261FF1F47
:103EF000FFFF0000293E001158BE0011EC40FF1FDB
:103F000000B50C4BBFB01A780B4902A800F0FCFCBE
:103F10006B4680B2D880002809D06A46074B01A9B9
:103F20001B889380064B0022188804F00BF83FB0E2
:103F300000BDC046A061FF1FA161FF1F4641FF1FDA
:103F40005042FF1F00B50C4BBFB01A780B4902A8B6
:103F500001F03EFF6B4680B2D880002809D06A4647
:103F6000074B01A95B8D9380064B0022188803F054
:103F7000E9FF3FB000BDC046CA61FF1FCB61FF1F14
:103F8000EC40FF1F5042FF1FF7B50E00377A1C00B0
:103F900008AB11003D001A8820231D401F423CD170
:103FA0003378022B3BD173681F785B781B023B434D
:103FB0001E4FBB4208D01E4FBB4214D01D4DAB421A
:103FC00021D00A252800FEBD002A2AD1142C2AD887
:103FD0002200F06807F068FD174B1C70012CF1D926
:103FE000FFF7B0FFEEE7002A1BD1202C1BD82200E0
:103FF000F06807F059FD114B04211C70104B187824
:1040000007F0B2FEDEE7E3B20124009201940A0059
:10401000310007F04BFB0500D4E70825D2E7012566
:10402000D0E70B25CEE70D25CCE7C046F3FF000017
:10403000F4FF000002290000CA61FF1FA061FF1FFA
:104040004C62FF1F332310B5040003700A22074996
:10405000013007F029FD064B0F201B681A0AE37296
:1040600022731A0C1B0E6273A37310BD1462FF1F20
:104070003C62FF1F30B5012503790400BFB02B421D
:1040800013D00B49408806F07DFE28420DD06A46C9
:10409000084B02A81B889380FFF7D4FF6B46D8809B
:1040A0000022608801A903F04DFF3FB030BDC0463B
:1040B000C261FF1F4641FF1F10B5024804F0C4FD56
:1040C00010BDC0467540001170B5160004AA1488D2
:1040D00005AA15784A685078117800022A4A0843E0
:1040E000801805284BD807F05FFC03131E29343FC6
:1040F0000720032C0BD80422121BAA4200D92A0045
:1041000022491A803000091907F0CEFC002070BD4A
:104110000720112CFBD81222121BAA4200D92A0018
:104120001B491A80EEE707200E2CF0D80F22121B35
:10413000AA4200D92A0017491A80E3E70720032C76
:10414000E5D80422121BAA4200D92A0012491A807B
:10415000D8E70720032CDAD80422121BAA4200D980
:104160002A000E491A80CDE70720032CCFD804225D
:10417000121BAA4200D92A0009491A80C2E700226C
:104180000A201A80C3E7C046DCD5FFFFA3BE00119A
:10419000E861FF1F93BE00118EBE001189BE0011A1
:1041A00084BE001110B50D21024A034806F062FDDD
:1041B00010BDC04678BE00115C41FF1F13B5104C06
:1041C0000423217C01AA00F0ADF9002815D16B462B
:1041D0009A88236852BA92B25343228909491B0C28
:1041E0009B184B806B46DA88636852BA92B253438D
:1041F00062891B0C9B188B8016BD0120FCE7C04612
:10420000FC61FF1F1462FF1F13B5124C06236A46A0
:10421000217C00F087F9002819D16B4619882368A2
:1042200049BA89B24B4321890B4A1B0C5B18538056
:104230006B46D97803335B781B020B435BBA61682A
:104240009BB24B4361891B0C5B18938016BD012008
:10425000FCE7C046FC61FF1F1462FF1F37B5174C17
:1042600007236A46217C00F05DF9002824D16B46C3
:104270001B787F2B20D86B46DD78F0232A041B03A4
:104280001A406B469B880E495BBA9BB21A4323685F
:104290002D09534322891B0C9B184B806B465A787F
:1042A0009B7812031B011A4363682A4353436289B4
:1042B0001B0C9B188B803EBD0120FCE7FC61FF1F9F
:1042C0001462FF1F7FB50226154C0022217C03AB30
:1042D0000096050000F0F8F8002802D0012004B094
:1042E00070BD0E23217C0122280000966B4400F053
:1042F000EBF80028F2D16B469A892368D2BA53436F
:10430000228908491B149B184B806B46DA89636825
:1043100052BA92B2534362891B0C9B188B80DEE722
:10432000FC61FF1F1462FF1F70B5184C237C002B2B
:104330000FD0382B0ED1164D280000F073F8CC2387
:10434000AC222800217C9B0100F027F9280000F016
:10435000A7F870BDE3890F4A934209D10C4D28009C
:1043600000F060F800222800217C00F005F9EDE75C
:10437000094A9342EDD1064D280000F053F89022EF
:104380002800217C920100F026F9DFE7FC61FF1F85
:104390003442FF1F830500008320000070B5144CD9
:1043A000237C002B1FD06369002B1CD0114D2800EB
:1043B00000F038F86369280098470400280000F0EE
:1043C0006FF8002C10D10C4B0422995E002905DAFD
:1043D0009C801A8801321A80200070BD074A9142E1
:1043E000F7DD9A80F5E70124FEF782FEF4E7C04688
:1043F000FC61FF1F3442FF1F1462FF1F0F270000E4
:1044000010B58024064AA4001168436B234205D1ED
:1044100013685B1A032BF8D9012010BD0020FCE7BC
:104420006008FF1F70B5C17905000C00631E9C4138
:104430001A4BE402E41849000460C9B2007906F09E
:1044400003F9E979687949000131C9B206F0FCF84D
:10445000E8790930C0B207F02FFB0023E36661332F
:104460002360AA795B3B002A0ED022689A43023B64
:10447000134323600A23E36107332362002323638A
:10448000A3630133E36370BD22689A43022313439D
:104490002360462363610633A361EFE700500040C9
:1044A00070B5002504000368DD66C0790930C0B22C
:1044B00007F0BAFA2900207906F062F8290060793D
:1044C00006F05EF870BD0000F8B51E0006AB1D7862
:1044D000002304681700E366616007F0F5FB012321
:1044E0008022E3662B0027615200013B08D207F0CF
:1044F00023FC08200A4A1168002D03D12800F8BDCA
:104500002261F2E7236F034203D02369013D337038
:10451000013613685B1A032BEED90125EEE7C0467E
:104520006008FF1F70B51C00002305681600EB66CD
:10453000696007F0C9FB01238022EB66230052006B
:10454000013B08D207F0F8FB08200A4A1168002C4A
:1045500003D1200070BD2A61F2E72B6F034203D024
:104560002B69013C3370013613685B1A032BEED9BB
:104570000124EEE76008FF1F002370B504681500F2
:10458000E366616007F0A0FB0123E366256107F0A5
:10459000D3FB2000FFF734FF70BD70B51D00002372
:1045A00004681600E366616007F08EFB0123E36692
:1045B00026610F33626B1A42FCD02B0A2361102351
:1045C000626B1A42FCD0EDB2256107F0B5FB20000A
:1045D000FFF716FF70BD002370B504681500E36691
:1045E000616007F071FB0123E3662B0A236110234E
:1045F000626B1A42FCD0EDB2256107F09DFB2000F2
:10460000FFF7FEFE70BD70B51E00002305681400A4
:10461000EB66696007F058FB0123A619EB660F33C0
:10462000B44205D107F088FB2800FFF7E9FE70BD12
:1046300021782961696B1942FCD00134F0E7000050
:1046400010B5084CE368002B08D18022064B5202BB
:104650001B689B186360054B1B68236007F09CFB7D
:10466000A06010BD3C62FF1FC8F00040CCF00040CD
:1046700070B5184A936A916A9942FBD116498A68C3
:104680009A421FD39A1A8B60144B0126186893B272
:10469000D202D20E4343424300204C681B0A1B192E
:1046A00012029B180E4C0A684B60551CA3420CD892
:1046B000002801D04B600A600A4A136008680A4B60
:1046C000186070BD581E821ADDE7084A30009B183A
:1046D0002A00EAE700F000403C62FF1F140AFF1FB7
:1046E00040420F00C8F00040CCF00040C0BDF0FFD9
:1046F00070B51F4C23793F2B01D93F2323711D4BEC
:1047000022791A701878C0B207F056FA18231A499D
:104710001A4A0B801A4913800B805380A3791949D8
:1047200080200B800C21938001334B43164D191CC4
:104730000001834200D9011C2980D1806379002BBC
:1047400001D101336371237A012B01D80223237233
:104750006279237A0D4853430A21584307F0C4F97C
:104760000B4D2860E379052B01D81023E37170BD50
:104770003062FF1F480AFF1F4E42FF1F1844FF1FF1
:104780004C42FF1F4A42FF1F4842FF1F71020000B8
:104790002062FF1FF8B520210020FEF761FE114CBA
:1047A000011E114D09D10C22104BC1CBC1C42800F0
:1047B00007F03AFAFFF79CFFF8BD0C2220000C49E5
:1047C000FEF722FE0C2802D0084B43CB43C40C2238
:1047D00028000849FEF718FE0C28EBD00C22002117
:1047E000E5E7C0463062FF1FFC61FF1F00BF0011FC
:1047F000FC0C0000F50C0000F0B51D4C8022A54417
:104800000400882069465201400507F0F5F990221E
:1048100012016A441300200032C832C316C816C3FE
:104820008023144C144FA6689B033343A3603B6062
:1048300007F0F2F88823A0685B05C01807F0CCF9F0
:104840000025882329008022A0685B05C018401934
:104850006944520007F058F880230135FF355B01A9
:104860009D42EED1A6603E60044B9D44F0BDC04623
:10487000FCEFFFFF8843FF1F9808FF1F0410000094
:10488000F0B5040087B0002825D0684607F0ECF8A2
:104890001B4C022806D106226946200006F084FF40
:1048A000002816D06946002301250F262F00E25C60
:1048B000013310091030874038002F0032409740F4
:1048C0003A0002434A610439062BEFD16846FFF7EC
:1048D00093FF07B0F0BD182269460A4807F08CF92B
:1048E0006A46A300D358013305D01822FF21684639
:1048F00007F09AF9EAE70134062CF1D1E9E7C0465E
:104900006509FF1F00090011F0B5002504000E0025
:1049100085B0AA4200D186E04B1C087801934B7801
:104920008978377909021943F3783F061B040B4352
:104930001F43039720706570252800D196E033D877
:10494000112813D806F018FF690037013701370125
:104950003701AA00B800B10037013701370137012C
:10496000370137013701370114013101232800D104
:10497000EDE0DB2800D040E1042A00D8B1E01025AA
:10498000052A05D0551F2A003800711D07F08CF844
:1049900005223100200007F087F82A003900601D49
:1049A00007F082F805353EE0562859D010D8332854
:1049B00000D1A7E0552839D02628DAD1A54B290007
:1049C000132218001D0007F02FF9FEF791FB5CE0A1
:1049D000712800D177E0722800D189E0602800D1E9
:1049E00095E0DC28C5D1022A00D87AE07378BFB2FE
:1049F0006370B378A370032A05D0033A390092B2EA
:104A0000F01CFEF73BFC10223900E01CFEF7FCFC1A
:104A1000C51C002807DA607070E00C2220008E4967
:104A200007F042F80C25280005B0F0BD013A8B4D87
:104A30000C2A13D8002A0AD02800019907F034F86C
:104A4000FFF756FE0C2228008549FEF717FC2900C7
:104A50000C22601C07F028F80D25E4E70C22EBE798
:104A60007E4D804B2A0043CB43C2E9E7013A794DA2
:104A70000C2A11D8002A08D00199280007F014F850
:104A80000C2228007849FEF7F9FB29001322601C4C
:104A900007F00AF81425C6E70C22EDE70622734951
:104AA000601C07F001F80625BDE712227049601C62
:104AB00006F0FAFF1325B6E708226E49601C06F0DF
:104AC000F3FF0925AFE7012A0ED07178F02908D845
:104AD000694D288801F0D8FD684B2A885200D35AC6
:104AE00000E0FF23637009E0634A644B1288F5E736
:104AF000634B012A04D072785A706270022592E7E3
:104B00005B78EFE72000FFF79DFA05008BE7013A9D
:104B10005C4D062A07D8002A06D1002301202B600D
:104B200001F09AF80CE006229621574B89001B6889
:104B300056485B1801992B6006F0B6FF01F058F853
:104B40000622601C691D06F0AFFF07256BE7042AEB
:104B500004D94D4D2F6007F01FF9A860FFF788FDBD
:104B60000422039003A9601C06F09EFF05255AE766
:104B7000474D062A15D906222800019906F014FE91
:104B800000280ED006220199280006F08DFF06228B
:104B900040492800FEF772FB0123394A51780B4344
:104BA000537006222900601CCDE7012A99D0707845
:104BB000FFF766FEA2E7012800D0DAE6931E364F23
:104BC000132B06D87378002B0BD100F019F900F0E5
:104BD0004FF9324B39001D78601C6A1E06F064FFE5
:104BE00021E7551E2A000199380006F05DFF3800C4
:104BF0002B49AAB2FEF742FBE9E7DA281DD1042AC5
:104C000000D86EE7082A15D9B37972791B021343CD
:104C1000F27912041A43337A1B0613433B603B6854
:104C2000052231002000039306F03EFF0422601DA0
:104C300003A944E7FE236370F1E7DE2800D050E7C4
:104C4000511E012A01D10025EDE6019800F0B6FFC2
:104C5000F9E7C046FC61FF1F0CBF00113062FF1F67
:104C6000FC0C000000BF0011F50C00000862FF1FE3
:104C7000E861FF1F8C43FF1F5042FF1FB064FF1FFE
:104C80002C62FF1F8C64FF1F3C62FF1F9164FF1F9B
:104C90006509FF1FADAC00002D64FF1F2B64FF1FD3
:104CA000AEDE000070477047020010B5094B0A32B3
:104CB000094C92B2DA815A8298811882207802F0E7
:104CC00049FB0422054B012120781A7007F04CF8AB
:104CD00010BDC0461643FF1F7664FF1F7564FF1F9B
:104CE000013870B5042809D806F05EFE03092808CB
:104CF0001200234B0221187807F036F870BD204BC4
:104D00000821187806F0F8FE00221E4B1A72F5E70B
:104D1000802200241B4B1A4D52001A8108211A6868
:104D20002878DC7206F040FF2100287806F014FF96
:104D3000012000F07BFE00F05BFFDFE7104B082155
:104D4000187806F0D9FE1048FFF71AF80F4B104AF2
:104D50009B79002093800F4A13808022094B5200D8
:104D6000D8721A8100F062FE00F042FF0A4B5B78B5
:104D7000002BC3D0094A136006F04EFDBEE7C046C3
:104D80004C62FF1F2062FF1F5942FF1F3062FF1F4E
:104D90001844FF1F4A42FF1F2C62FF1F34F00040DF
:104DA00010B500290BD1082809D1054B1B78002B21
:104DB00005D02622034B04485A72FFF775FF10BD39
:104DC0004E64FF1F2062FF1FC40900000300F0B5FE
:104DD0000A4D8E18B14202D152008018F0BD0C78F5
:104DE0002F6824093C5D0F271C700C7801313C4072
:104DF0002F683C5D5C700233ECE7C0464442FF1F05
:104E00000D22124B10B51A700C23114C114923704E
:104E1000093A033B1048637006F046FE2D23012239
:104E20000E490F48A371FFF7D1FF01220D49FFF78B
:104E3000CDFF01220C49FFF7C9FF030000200B49F9
:104E400002001870FEF71AFA10BDC0464A64FF1F30
:104E50002B64FF1FA3BE00112D64FF1F6709FF1FF6
:104E60003264FF1F6609FF1F6509FF1FAEDE0000E9
:104E700070B5134C142220001249FEF7C5FA431EE8
:104E8000114D132B19D8AB78002B16D0431C2B7067
:104E900009236B7000230019037028780B4B013035
:104EA0002900C0B2187006F057FD29782200013998
:104EB000C9B2002005F0FCFD70BDFFF7A1FFECE7D3
:104EC0002D64FF1FAEDE00002B64FF1F4A64FF1F2E
:104ED00010B5114B1A781870002A0ED000280BD18B
:104EE0000E4B1A78062A07D85423D340DB0703D584
:104EF0000B4B187802F02EFA10BD0028FCD0074B9F
:104F00001B78012B02D0033B022BF5D8044B012167
:104F1000187806F029FFEFE74E64FF1F7564FF1F46
:104F20007664FF1F70B5514E514A524930700820C7
:104F300005F04AFC0121022005F050FB022005F09B
:104F400031FC0121002005F049FB002005F02AFC7E
:104F500000F0DAFEFEF7CCF806F01EFD032246490B
:104F60004648FFF733FF2D24030004221C704449F8
:104F70000130FFF72BFF30230470424D424C437049
:104F800083702E3B062220004049EB87FEF73CFA57
:104F9000062813D0200006F067FD022809D003215F
:104FA000200006F069FC8D23E3706E3B23711933FA
:104FB0006371062220003549FEF760F9344B1B6807
:104FC000FC335C64FFF754FF0020FFF781FF314C96
:104FD000314A0121314B1278207802F07DF9304AB4
:104FE000304B12780021207802F076F901222E4B06
:104FF0001A702E4B9B78552B31D12D4B3B325A7268
:105000002C4B2D4AAB81EA812B826A822021307899
:1050100006F062FE0120404205F096FD012040426C
:1050200005F032FEFFF7BEF8FEF772FE00F0B2FCAC
:1050300001204042FEF748FF012006F015FEF02057
:1050400001F006FB0121307806F08EFE307802F088
:10505000DDFA1A4806F098FBFEF708FD70BD6422E1
:10506000174B5B7953431A000A32CBE74C62FF1FA0
:10507000A14D0011A54C00118C43FF1FE861FF1FDB
:105080000862FF1F1643FF1F6509FF1FADAC00003C
:10509000AC64FF1F7664FF1F7842FF1F5942FF1F59
:1050A0004A64FF1F2B64FF1F1C64FF1F2C62FF1F3D
:1050B0002062FF1FC4090000CE0900004E62FF1FDE
:1050C0003062FF1FF8B50A0020230D001A40194274
:1050D00063D05E4B1B78002B5CD0FFF7C9FA5C4BAA
:1050E0005C4C5D4E99686268737A8A1ADB039A4257
:1050F00002D36160FEF7BAFC327A217A531EDBB22A
:10510000994205D1FFF710F9002000F0A5FD15E048
:105110009142F9D300272772FFF740F9A37ABB42E7
:1051200002D0A772FEF730FD012000F095FD4B4F35
:105130003800FEF725FE390006F0DEFB637A002B0F
:1051400025D0013BDBB26372002B20D1444B9B780E
:10515000552B01D106F060FBE37A002B12D000231F
:10516000A27AE3729A4202D0A372FEF70DFD3D4A85
:105170003A4F1388380001331380FEF701FE3900DF
:1051800006F0BAFB642370795843FFF78DFD237A4C
:105190000133237220206840F8BD0BB2002B0ADADD
:1051A000314B187806F030FD002801D006F0E4FC01
:1051B00080200002EFE70224214206D0254B012087
:1051C0001A72FFF785FE2000E5E70B071ED5FFF7F3
:1051D0004FFA1F4B1F49204C98684A68637A821A1D
:1051E000DB039A4202D34860FEF740FCFFF7D6F893
:1051F000FFF79AF8012000F02FFD00F0E5FB23688F
:10520000DB0701D5FEF758FF0820C4E7CB0609D518
:10521000FEF7BAFC0D4B1B78002B01D1FEF78CFD7D
:105220001020B8E70124214207D0104800F06CF8A4
:1052300006F09AFB00F0F6FCC5E7042408002040C5
:105240002142A9D0FEF75CFEBDE7C0464E64FF1FB9
:105250003C62FF1F2062FF1F3062FF1F5942FF1F89
:105260002C62FF1F1462FF1F4C62FF1F3C42FF1F96
:10527000F0B51B4B1B4F1B883A8804001A4E1B4D80
:1052800085B09A420DD832889A420AD3184B1A88B0
:105290002B889A4205D1174A174B12881B889A42CD
:1052A0001BD0052001F02AFA3B8802AA138033881C
:1052B000019053802B88114D93800F4B02A91B88BE
:1052C000D3800F4B2A78188802F046FF0D4B082137
:1052D0002878019A1C7006F037FB05B0F0BDC04677
:1052E0001A64FF1F4E42FF1F4C42FF1F4A42FF1F1E
:1052F0001864FF1F1664FF1F4842FF1F7664FF1FDC
:105300005042FF1F1464FF1F13B50C4B1C78002C78
:1053100011D1002801D00A4B18600A4A0A4B1178B3
:105320000A4A10780A4A01920A4A0092002205F0BD
:10533000B7FA200016BD1124FBE7C0467564FF1FB5
:105340001064FF1F7464FF1F6464FF1F7664FF1FF7
:105350005064FF1F5464FF1F10B5064B12201B78CA
:10536000052B06D1044B13221988044B187801F041
:10537000A1FB10BD7564FF1F5042FF1F7664FF1F25
:1053800010B500240122114B52421870104B1C70B2
:10539000104B1A8002F03AF904220F4B21001A70C8
:1053A0000E480C3206F0B8FC102221000C4806F022
:1053B000B3FC07220B4B1C600B4B1C700B4B1C707F
:1053C0000B4B1A700B4B1C7010BDC0467664FF1F50
:1053D0007564FF1F5042FF1F7464FF1F6464FF1F4A
:1053E0005464FF1F5064FF1F2A64FF1F2964FF1FBE
:1053F0005242FF1F2864FF1FF8B5174C060025789E
:1054000006A814240078052D23D1B41F134FA5B28C
:105410001824BD421DD88D1FADB2BD4219D8FA2542
:105420006D00AA4215D21D000D4F0A3DADB2BD421E
:105430000FD80C4C26800C4C21800C4900240A808B
:105440000B4A1380FFF714FF0A4B0421187806F06B
:1054500053FB2000F8BDC0467564FF1F790C0000A7
:10546000750C00004E42FF1F4C42FF1F4A42FF1FB7
:105470004842FF1F7664FF1FF0B50BB20D0089B0E4
:10548000002B00DB70E1A44E307806F0BDFB041E5B
:1054900050D00378A22B00D122E1D02B1AD0912B2F
:1054A00045D143780E2B42D19C4B82889A423ED103
:1054B0009B4A83681278052A39D1032018567F2821
:1054C00035D0984B1B68002B31D05B68002B2ED059
:1054D00098472CE08078072829D806F065FA042838
:1054E000183F3F74A8D86378002B0CD101218C4B56
:1054F00019708D4B1A78002A5BD08C4B307801F0F4
:10550000EBFE002855D00722854B1A7051E06178D8
:105510000029F8D1E378002B11D0854A854B127809
:10552000307801F0D9FE60706378002BEBD1200059
:1055300006F022FB80200002684009B0F0BD784BE5
:105540001B78022BF3D00121307806F095FA002861
:10555000EAD10121307806F007FCE5E76378002BFB
:10556000D1D16F4F032807D13B78052B02D10133EE
:105570003B701EE00223FBE76F4B1A886F4B0293D0
:10558000002A0BD01B78002B03D00121307806F0C5
:10559000DBF93B78062B04D1013BE9E7029B1A704B
:1055A000F7E7042B41D10121029B3078197006F0F6
:1055B000DBFB5C4B1B68002BB9D01B68002BB6D003
:1055C000574A107884E76378554F002B27D106227D
:1055D000211D5B4806F068FA62895A4B5A491A80C5
:1055E000A2895A4B1A80E3890B80052139705849EA
:1055F0000A80584A1380228A574B1A80574B1B78CF
:10560000012B09D11F2001F079F8FA2292004243C0
:105610000421307806F098F90022484B75E7312BC9
:1056200000D070E70022454B1A700323A0E7062242
:105630000021434806F070FB0023454A04211380F3
:10564000444A30781380444A138006F055FA082102
:10565000307806F051FAA379083B5A425341304A58
:1056600003331370304B1B78002B06D0334B30784C
:105670001A78002A06D001F06DFE0122314B524209
:105680001A8096E70121197006F06EFBF5E70821F4
:10569000307806F031FA6378002B00D047E72C4BC6
:1056A0002D4F0293E388029A04211380294B30780E
:1056B00003932389039A138063893B8006F0DCF906
:1056C000002800D033E7264B1B68002B00D12EE7C3
:1056D000039902983A88098800881B68984726E74A
:1056E0004379132B00D022E70389012B0AD11D4BEC
:1056F0001B78022B06D10821307806F0FDF9FFF760
:105700002BFE14E7052000F0F9FF08210200307895
:1057100006F01AF90BE7C0467664FF1F0514000077
:105720007564FF1F1064FF1F7842FF1F5942FF1F5F
:105730004A64FF1F2B64FF1F4C64FF1F4E64FF1F52
:105740001D64FF1F5042FF1F2464FF1F2664FF1FBC
:105750001A64FF1F1864FF1F1664FF1F1C64FF1FDD
:105760000C64FF1F1464FF1F8020C001014200D0A1
:10577000E2E6CB0731D5324B1B78002B1DD0314EE2
:1057800005AC3378052B1AD1023B23702E4B210038
:105790001B7823722D4B1B7863722D4B187801F008
:1057A0003FFD002809D007202A4B30701B68002BD2
:1057B00003D01B68002B00D098470120BCE60E20C8
:1057C000254B06221B7825492370254B1B786370D7
:1057D00002ABC01806F068F9D8E7022308001840A9
:1057E000194209D0174B1B78052B03D11D4B188884
:1057F00006F072F802209FE60424214203D0FFF74E
:1058000037FD200098E6082308001840194200D10F
:1058100093E6154B1C78012C03D0022C0DD00820E8
:105820008AE6124B124A134913481B8812880988CA
:1058300000880094FFF7E0FDF1E7FFF78DFDEEE74C
:105840004E64FF1F7564FF1F5242FF1F2864FF1F35
:105850007664FF1F1064FF1F2A64FF1F5342FF1F5F
:105860002964FF1F5042FF1F1464FF1F4842FF1F9F
:105870004A42FF1F4C42FF1F4E42FF1F10B502A8B5
:1058800004880B20002C10D1496808784978090257
:1058900001430C48814209D1022119800A4B5988E1
:1058A0001170DB7800205BB2537010BD074C0A20EA
:1058B000A142FAD102211980034B998811705B79BA
:1058C000F0E7C0466E2A00001462FF1F6F2A000036
:1058D000F7B5150008AA16884A680F4F1478527851
:1058E000120222430A24BA4214D10122DBB20192ED
:1058F00000962A0005F0DAFE041E0BD1074B1B6848
:10590000002B07D068782A780002104342425041A9
:10591000013098472000FEBD022900008864FF1F67
:1059200030B5012503790400BFB02B4225D01449BE
:10593000408805F027FA28420CD0124B01A95B8D54
:1059400000220B8002234B800F4B5B888B8060888A
:1059500002F0F8FA0D49608805F014FAC0070CD57A
:105960000B4B01A91B8800220B8002234B80064BA6
:105970009B888B80608802F0E5FA3FB030BDC0465E
:105980008064FF1F7C42FF1F1462FF1F7864FF1FAB
:10599000D642FF1F10B5074C0749200005F0A8F9B3
:1059A0002000064905F0A4F90721054A054805F03D
:1059B00061F910BDFFFF00008064FF1F7864FF1FC6
:1059C0002CBF00117C42FF1F10B5024803F03CF9C8
:1059D00010BDC0462159001170B55F250826074942
:1059E00084000A7ACB7940012A40B3433440A8436B
:1059F00023430243CB710A7270BDC0468C64FF1F03
:105A0000010043B204205A0002409B000C300340C6
:105A10001A43152310B5044C207A9843143B0B40CD
:105A200018430243227210BD8C64FF1F10B5054B52
:105A30000824597A0A00A243002801D022000A4310
:105A40005A7210BD8C64FF1F10B5054B4024197AA3
:105A50000A00A243002801D022000A431A7210BD96
:105A60008C64FF1F0821F8B5324D334BEE790400EA
:105A70000E40EE71984204DD67236B71473BAB71BA
:105A8000F8BD2E4B984203DAE0236B713A3BF6E700
:105A900000236B71AB7183B21A0029485F3292B256
:105AA000284F82422CD9002C03DA5B421CB204231B
:105AB0006B71053420B20A2106F016F804B2FA23FD
:105AC0009B009C4232DB08236A7913436B7164218B
:105AD000200006F009F80A2100B205F0BDFF09B266
:105AE0006A797B5C13436B710A21200005F0FCFF8F
:105AF0000A2100B205F0B0FF09B27B5CAA790AE086
:105B0000A971002CDBDA5B421CB204236B71F32217
:105B1000AB79092CE8DC1343AB710A21200005F0B6
:105B20009BFF09B27B5C1E43EE71A9E7632CCEDCC0
:105B3000EDE7C0468C64FF1F1B4E00001DFCFFFFFD
:105B40002A08000056BF00110823F7B5194FCD00F1
:105B50007E7A04001E407E72EDB2632806DD5F335C
:105B600033437B7220231D43BD72F7BD030009330D
:105B700005DA20235B4233437B72A623F3E70E4B07
:105B8000019300280BDA0423444224B27B720A21D9
:105B9000200005F061FF019B09B25B5CE3E7092887
:105BA000F5DD0A2105F0A0FF019B00B21B5C1E433E
:105BB0007E72ECE78C64FF1F56BF0011F8B50A4FE8
:105BC00005003B790E00002B0CD0084C2000FEF79E
:105BD00029FC33002A0020003979FEF714FD20004B
:105BE000FEF75EFCF8BDC0468C64FF1FF042FF1F4D
:105BF00070B5094D094C06222900200005F0D4FD9E
:105C0000002808D029000622200005F04DFF0721BA
:105C10000348FFF7D3FF70BD9164FF1F9864FF1F17
:105C20009764FF1FE622402110B5094B5A71094ABB
:105C3000DA801A7A0A401A720822597A1140533AC5
:105C40000A435A72F3229A72FFF7D2FF10BDC04680
:105C50008C64FF1FA6E4FFFF254A264B12681B68D1
:105C600010B59A423AD3002838D0234C0223E05E84
:105C7000224B1B685B0632D509233221584305F0BD
:105C800033FF4130FF3000B2FFF7ECFE0520FFF795
:105C9000A3FE0422A35E1A4A6320934205DC32333A
:105CA0001800642105F020FF00B20121FFF74CFF2E
:105CB000237A0024132220009A426041C0B2FFF7E9
:105CC000C3FE2000FFF79CFE0E4B187805384342B8
:105CD0005841C0B2FFF7AAFEFFF78AFF10BD0A21A4
:105CE000053005F001FF00B2FFF7BCFE0320CEE750
:105CF0003C62FF1F8C64FF1F1462FF1F3062FF1F96
:105D0000DD2600007564FF1F70B500250A4C2000D9
:105D1000A571FEF787FB10233E212000074AFEF7FE
:105D200072FCA84200D13E35054B20001D71FEF7E4
:105D3000B7FB0123A37170BDF042FF1F46BF0011E6
:105D40008C64FF1F0200F0B501270A480A4E511863
:105D50008B1A002B00DCF0BD08241578430868403E
:105D600038404000805B013C58406D08002CF5D164
:105D70000132EDE7FFFF000066BF0011F0B500251E
:105D80000F269D4200DBF0BD4C5D070944403440C6
:105D9000A400A05801357840F3E70000F0B589B0C1
:105DA0006A460D000B000F27110010351C780133D7
:105DB000260024093E40167054700232AB42F5D1E1
:105DC0002023024AFFF7DAFF09B0F0BD6CBF0011D3
:105DD000F0B54E780B7889B036020C0017000190B0
:105DE0001E43012A61D9954B9E4200D877E00133CA
:105DF0009E421CD1062A17D1CA788B7812021A4308
:105E00000B791B0413434A7912061A438C4B5A61CF
:105E100000221A705A808B4A5A608B4A9A608B4AC9
:105E2000DA60002009B0F0BD88225205EEE7884B09
:105E30009E423CD182498B78002B00D0F6E00C2AA0
:105E400031D10F22A3789343E278120213432279CF
:105E5000120413436279120613434B60E279A0796E
:105E600012020243207A00041043627A12060243AF
:105E7000CA60E27AA07A1202024376484A818342DB
:105E800008D804236E49142201980B7005F00CFE0B
:105E90001420C7E71201D21889235B059A42F0D873
:105EA00001238B70BDE7022AFAD00523EAE76A4A8C
:105EB00001239642E6D1FFF74FFA052F0CD9E3787C
:105EC000A2781B021343227912041A4363791B063A
:105ED0001343624A0393136005F09EFCA1E7584DFB
:105EE0002B78002B9DD1AB78002B00D1A0E02B8923
:105EF00001339BB20093B34200D091E0132AD4D96E
:105F0000CF7C8B7C3F02122120001F43FFF71AFF3A
:105F1000874200D08EE0002E3DD1E378A2781B02AC
:105F200013432279E96812041A4363791B06134369
:105F300003930A228B4212D1FF23A370E3702371D3
:105F400063716B89002B09D1E37B227C1B02120455
:105F50001343A27B13431B0901336B8100226B891E
:105F6000002B8ED0002A67D1686837013818000BE3
:105F70006B6900030390984205D9686105F02CFE17
:105F8000EB780133EB7068681022A11C381805F01B
:105F9000BBFC2E8145E76F89009A7B1E9BB2934222
:105FA0003AD1E278A37812021A43237905A81B0498
:105FB000134362796C6812061A43EB6800920392ED
:105FC000211D0C22049305F06FFD0120260004A979
:105FD00040421036FFF7E2FE013F012F17D1009A31
:105FE0000B232861824200D04CE704221C49200088
:105FF00005F08AFC042203A9686805F0FDFDE96844
:10600000039AFF23914200D13CE7F73B3AE7310086
:10601000FFF7C4FE1036DFE70923B742A4D831E703
:10602000009BB34200D9FCE607232BE7022329E7B4
:10603000032327E7062325E70A2323E7FFFE0000C3
:10604000F842FF1F00000111FFFF000050485936C1
:1060500001FF0000FFFF001102FF000034F00040CC
:106060000443FF1F10B5034C0B000122210000F078
:106070006BFA10BD256200110B8870B506000D008B
:106080000224162B11D92B000322094900F05CFAD7
:10609000041E0AD1074B2A881B88191C934200D979
:1060A000111C300089B200F0EFFA200070BDC0462C
:1060B00051620011B264FF1F10B54A780400013A22
:1060C0000B000220012A07D80A78002A04D00522F2
:1060D0002000024900F038FA10BDC0467F6200116E
:1060E0000A7810B50B0004000220002A04D0072211
:1060F0002000024900F028FA10BDC0462B630011B1
:106100000A7810B50B0004000220002A04D00922EE
:106110002000024900F018FA10BDC046916300113A
:1061200010B5034C0B000B22210000F00DFA10BD3E
:10613000C163001110B5034C0B000D22210000F0CB
:1061400003FA10BD3364001110B5034C0B000F228D
:10615000210000F0F9F910BD8D6400110A7810B526
:106160000B0004000220002A04D011222000024962
:1061700000F0EAF910BDC0469D640011002310B57F
:106180001322190000F0E0F910BD000010B5034C17
:106190000B001722210000F0D7F910BDEF640011A9
:1061A000002310B51922190000F0CEF910BD00002F
:1061B00010B5034C0B001B22210000F0C5F910BDE7
:1061C00029650011F7B584890D0006000121002C16
:1061D00022D000238268D3561778002B1EDA0C2CAD
:1061E0001AD90C3CA4B2131940880093230002F082
:1061F00086FE431E984101307B06DB0F6B703F2308
:10620000013C1F40A4B22870AF70AC80002C07D0B6
:10621000B3680133AB6000210800FEBD0020EBE74E
:10622000AC60F8E70B7803704B8843704B881B0A0F
:1062300083700B79C370042070470420022B06D1B1
:106240000020537811781B02009A0B43138070478B
:106250000B8803700B881B0A4370022070470420D0
:10626000009983420AD1537810781B0203430B80B4
:10627000D37890781B02034300204B807047F8B519
:106280000D004B7801240021461C03702B788B42B3
:1062900001D82000F8BD6B78B01C4F1C012B10D129
:1062A000890069184B88022233704B88B9001B0A99
:1062B0007370691805F0C8FA04360434A4B2F9B250
:1062C000E4E7122359436B185A88043132705B8813
:1062D00010221B0A7370691805F0B6FA12361234D0
:1062E000ECE770B5049D14001E00052B01D80420B6
:1062F00070BD637812781B0213432B80E378A27879
:106300001B02134302226B802A71211D681D063E69
:1063100005F09AFAB2B22A81E92AE8D82800A11D2C
:106320000A3005F091FA0020E2E7002310B50A7860
:106330009A4201D8900010BD9A008A1854880133FF
:1063400004705488DBB2240A447094888470928864
:10635000120AC2700430EAE710B51100029C062B45
:1063600004D004201022142B01D010BD022222716F
:106370004B7808781B0203432380CB7888781B0274
:10638000034363800431601D05F05EFA0020ECE7F2
:1063900010B50C788B7804315C43E4B203702200B2
:1063A000013005F051FA601C10BD0420022B06D10B
:1063B0000020537811781B02009A0B43138070471A
:1063C00010B50C000A88023105F03EFA208810BD95
:1063D00070B504000D0004981100012B01D80420B1
:1063E00070BD167852781202324302800200F132F8
:1063F00055701470E125002C00D10C35023B9AB287
:106400004280AA42EBD80231043005F01DFA002088
:10641000E6E70420009983420AD1537810781B02E2
:1064200003430B80D37890781B02034300204B80FA
:10643000704710B50C000A88023105F005FA208873
:1064400010BD000070B501211E000420049C0E4008
:106450000B4218D1CB40DDB28D4214D90A49DBB2D0
:10646000098899420FD32300EE331D703300580082
:1064700011184978165C0902314301332152D9B20F
:106480008D42F4D8002070BD1043FF1F10B50C00E2
:106490000A88023105F0D8F9208810BD10B50C78B3
:1064A0008B7804315C43E4B203702200013005F0C4
:1064B000CBF9601C10BD10B511000298032B01D858
:1064C000042010BD14785278043B1202224302804B
:1064D000CA788C781202224342809AB28280EB2AD8
:1064E000EED80431063005F0AFF90020E9E710B529
:1064F0000C000B8803700B881B0A43704B88837059
:106500004B881B0AC3708A880430063105F09CF959
:10651000A088043080B210BD0420012B03D10020DC
:106520001378009A1370704710B50C000B88037035
:106530000B881B0A43704A880230043105F084F945
:106540006088023080B210BDF0B589B003931E4B55
:10655000029242000700D05A019102F020F8132560
:10656000061E2DD0029B01240370019B002B04D03A
:10657000001903999847001984B26B461B7A5BB2E5
:10658000002B0FDA1021380002F01CFB192500281F
:1065900013D130003219E1B202F066FC051E0CD1B5
:1065A0000C34A4B2042304AA380005A993800696EB
:1065B000948101F0AFFD051E02D0300005F024FAF1
:1065C000280009B0F0BDC046B064FF1F70B50500DB
:1065D0000C0000280CD00020814209D0102220009D
:1065E000044905F031F901202B7823736B7863732C
:1065F00070BDC046ACBF0011F0B506000D0017001D
:106600001C0085B002291BD00020102907D1022BC5
:1066100007D0102B03D115E00020102C08D005B0B6
:10662000F0BD69463800FFF7D1FF2A0069460BE04C
:1066300069463000FFF7CAFF22006946380004E0CF
:10664000022BE9D12A003900300005F025F9E6E7F0
:10665000031CF02800D9F023032008499AB2013A1C
:106660000B80D317034006499B189B100B80D30F58
:1066700004499B185B100B807047C0461443FF1FF2
:106680001243FF1F1043FF1F034B1B888B4202D393
:10669000024B4000C15270471443FF1FB064FF1FFC
:1066A000014B4000185A7047B064FF1F1722014B7E
:1066B0001A807047B064FF1F70B505000E2005F00A
:1066C000E3F9041E13D0D023037000230622837045
:1066D00007494570033005F0B7F8064B2100DA8A08
:1066E00062811B7E2373044B187805F085F870BD1A
:1066F000CC64FF1FBC64FF1F6443FF1F262803D820
:10670000024B4000C05A70470148FCE71643FF1F88
:10671000FFFF000070B506000C00094D1C2200218F
:10672000280005F0F9FA074B1E70074B1C7005F0A6
:10673000C3FA0123002801D0002312202B7070BD62
:10674000BC64FF1F6443FF1FDD64FF1F70B50500BD
:106750000D4C0800E260A16010220021656005F088
:10676000C3F8012803D11021A06802F058FD1022BF
:106770000021280005F0B8F8012803D11021606835
:1067800002F04DFD70BDC046BC64FF1F70B5041E15
:1067900005D1002903D006220D4805F055F80D4B10
:1067A0001D78012D11D1002C05D102221A7005F09F
:1067B0009BFA280070BD00221A70074B1B78FF2B34
:1067C000F7D02000FFF778FFF3E70025F1E7C04698
:1067D000CC64FF1FBC64FF1F6443FF1F030010B5A0
:1067E000002801D1002010BD00780B4A002803D1F9
:1067F0005988D1821B7913761378022BF2D10023AA
:10680000984200D103331370044B1B78FF2B01D047
:10681000FFF752FF0120E6E7BC64FF1F6443FF1F40
:10682000002911D000280CD04B79012803D1402237
:106830005242134303E03F221340032802D00120B9
:106840004B7170474022F4E70800FAE770B5094D34
:106850000100287800280BD0074C0622200004F005
:10686000F3FF21002878FFF7DBFF200005F02CF86C
:1068700070BDC046DC64FF1FB664FF1F00290AD04C
:10688000012808D13F224B799343C02B03D0403BD2
:106890005A425341981C704770B5174D06002B782B
:1068A000FF2B15D00A2005F0EFF8041E10D0D023DE
:1068B0000370C83B8370114B11491B784670C3703D
:1068C0000622043004F0C0FF2100287804F094FF71
:1068D0000C4B1B78012B0DD10B4B1B68002B03D0ED
:1068E0009B68002B00D09847084B04211878084A71
:1068F00005F05AF970BDC0466443FF1FDC64FF1FFA
:10690000B664FF1FD864FF1F0465FF1F0865FF1FE3
:1069100060EA0000014B98687047C046BC64FF1FE6
:10692000014BDB6818687047BC64FF1F074B10B54C
:10693000DA68136801331360054B1878FF2803D019
:106940008021C90105F010FA10BDC046BC64FF1FCC
:106950006443FF1FF7B50E0002F0C8F8051E1CD0F7
:106960000E4B06621F78002F00D10778AB791020FC
:10697000019305F089F8041E0FD0D0230380C73B94
:106980008370019BE91DC3700622043004F05CFF94
:1069900021003800E66004F02FFFF7BD6243FF1FBF
:1069A000014B18787047C046DC64FF1F054B002878
:1069B00005D1054B1A78054B002A00D1014B180070
:1069C0007047C046CC64FF1FDC64FF1FB664FF1F26
:1069D000014B58687047C046BC64FF1F024B1868E3
:1069E000431E9841C0B27047E064FF1F421E03007F
:1069F0000120152A03D9FF3B5A425341D8B27047B0
:106A0000F0B51C0000230E0085B0039002920B70BD
:106A1000029A934201D3002019E0E55C5A1CD2B2DD
:106A2000002DF8D0029851198142F4DC0233DFB214
:106A3000A35C18000193FFF7D9FF002807D0013DA0
:106A4000019A0399EBB233708A4202D1E01905B082
:106A5000F0BDDB19DBB2DBE710B50C0002F09EF8ED
:106A600003001220002B03D02100588804F0BCFE44
:106A700010BD000070B50E4D84006359002B15D079
:106A8000186A002801D005F00FF92B59586A002820
:106A900001D005F009F92B59986A002801D005F0BA
:106AA00003F9285905F000F900232B5170BDC046A9
:106AB000EC64FF1F1C4B70B504000E0015009942DA
:106AC0000AD11A4B1B68002B01D1122070BD1B6824
:106AD000002BFAD09847F9E7154B994215D1134B83
:106AE0001B68002B0AD01B68002B07D09847002892
:106AF00004D1104B1C70104B1D70E7E729002000DB
:106B0000FFF7AAFF0028E1D1F3E7080001F0EEFF4C
:106B10000028DAD003780320A342D7D1290030001F
:106B200004F062FED2E7C046FEFF0000E864FF1FEB
:106B3000FFFF0000E564FF1FE464FF1FF7B50400DA
:106B4000808801F0D3FF0025A84203D00578A088F3
:106B500002F008F81C4E3378002B1FD0AB421DD139
:106B60001A4B28001978FFF777FF002818D0002368
:106B70003370A3790820A778A688019304F084FFD6
:106B8000011E0DD0D0230370CA3B8370019B477058
:106B900086808371280004F02FFE01E0002DE8D1EB
:106BA000A0880B4B8200D358002B01D0FFF762FF67
:106BB0001721A088FFF768FDA08801F027FDA088B5
:106BC00001F0FEFDF7BDC046E564FF1FE464FF1F52
:106BD000EC64FF1FF0B587B01D000CAB1B880700ED
:106BE00001930DAB1B88142002930EAB1B8816007B
:106BF00003930FAB1B880091049310AB1B88059384
:106C000004F042FF041E1AD0D0230370CB3B477020
:106C10008370C670062229000430002D11D004F0C4
:106C200013FE019B21006381029B0098A381039BBB
:106C3000E381049B2382059BA37404F0DDFD07B070
:106C4000F0BD05F069F8ECE7F7B5009308AB1B88D9
:106C500007000C200D001600019304F015FF041E20
:106C600013D0280001F042FF00280FD00078D02375
:106C70002370C93BA370009B21002381019B677097
:106C8000A580E680638104F0B7FDF7BD014B18785D
:106C9000EDE7C0466443FF1F13B504006489038910
:106CA000C2888188C0780094FFF7CEFF13BD000032
:106CB00010B5044C2068002803D004F0F5FF002331
:106CC000236010BDF064FF1FA122F0B581889200FF
:106CD0004A43384B384F1B6804009B189D22920092
:106CE0009B18827989B01A603B68002B5FD01D78B1
:106CF000324B1B68002B04D05B68002B01D00020B6
:106D00009847260008363100E079FFF7B7FD237D6C
:106D1000E0710200E0780493638A29000393238AD8
:106D20000293E3890193A38800933300FFF752FF96
:106D3000E378002B0BD1E289A379A1880292019616
:106D4000E27928000092012201F0DAFEE0703B684F
:106D5000002B20D0FFF7ACFF194D287800281AD05F
:106D6000184B1978FFF778FE002814D02B78E678B6
:106D700008200793A78804F087FE011E09D0D023BE
:106D80000370CA3B4670837087808671079804F051
:106D900033FD00232B701721A088FFF775FCA08816
:106DA00001F034FCA08801F00BFD09B0F0BD064BEA
:106DB0009DE7C0463409FF1FF064FF1F0465FF1FF5
:106DC000E564FF1FE464FF1F6443FF1FF8B507007D
:106DD00008000E0001F08AFE041E18D02620FFF7DE
:106DE0008DFC051E00D12578062004F04DFE041E02
:106DF0000DD00021062204F08FFFD0232370C23B68
:106E000021006770A370A680E8B204F0F5FCF8BD1D
:106E1000F0B585B001930AAB1B78070002930BAB6A
:106E20001B7808000D000092039301F05FFE061E20
:106E300022D0102004F028FE041E1DD010220021B4
:106E400004F06AFF2620FFF759FC002800D13078B3
:106E5000D0232370C13BA370009B21002372019BB0
:106E600067706372029BA580A372039BC0B2E3723A
:106E70000C9BE36004F0C0FC05B0F0BDF7B50D005D
:106E8000019001F033FE071E20D00E2004F0FCFD1F
:106E9000041E1BD02620FFF731FC061E00D13E78D1
:106EA000D0232380C53B0622A370F91DE01C04F00B
:106EB000CBFC019B2A0063810123DD401A401D4069
:106EC000210022736573F0B204F096FCF7BD000058
:106ED000F0B585B0029010000D0017000A9E0393D4
:106EE00001F004FE041E31D0029B002B2ED1039B27
:106EF00002795B0724D5122313430422002E08D104
:106F00000B99002905D10C99002902D10D9900296E
:106F10001AD01A430D9B2271002B00D0C9E0002E1D
:106F200000D1CFE0002D00D0CCE0606A002801D075
:106F300004F0BAFE1C21300004F07EFE606205E021
:106F400002239A430E33D7E793432371654BBA006C
:106F5000D458002C00D1AAE0002E10D0236A002BB8
:106F600003D11C2004F010FE20625E4BBA00D358FF
:106F7000186A002803D01C22310004F065FC0C9B29
:106F8000002B12D0574CBB001D596B6A002B03D14C
:106F9000162004F0F9FD6862BB00E358586A002827
:106FA00003D016220C9904F04FFC0D9B002B11D03E
:106FB0004C4DBC006659B36A002B03D1142004F079
:106FC000E3FDB0622B59986A002803D014220D9972
:106FD00004F03AFC380001F089FD051E67D0414BF2
:106FE000BA00D358002B62D01A6A3420002A00D18C
:106FF0001C389A6A002A01D0143080B20B9A002AF9
:1070000001D01C3080B25B6A002B01D0163080B2F8
:1070100004F03AFD041E4AD01822002104F07CFE40
:107020002620FFF76BFB0190002801D12B780193FC
:10703000D0232370029B200063700A23294EA37083
:10704000039BBD00A371AB59A780196A18300029B2
:1070500005D01C22A06004F0F7FB200034307359E7
:10706000996A002907D0030014221433E0600293C8
:1070700004F0EAFB02980B9B002B08D003001C22B3
:107080001C330B992061029304F0DEFB02987359C4
:10709000596A002903D01622606104F0D5FB6B46C3
:1070A0002100187904F0A8FB3800FFF7E3FC05B0D5
:1070B000F0BD10220D9B0D991B69A018236204F0EE
:1070C000C3FB2CE70B9B002B00D13FE7012D00D029
:1070D0003CE7606A002801D004F0E6FD1C210B9813
:1070E0002AE7C046EC64FF1F10B5044C2068002856
:1070F00003D004F0D9FD0023236010BDE064FF1F1E
:107100000B4B07B51A68002A01D100200EBD694655
:10711000531C012012780731FFF772FC0028F4D0CD
:1071200002780123100018401A42EED0EEE7C04664
:10713000FC64FF1FF0B51F4F01203B6887B0002B98
:1071400025D09B78059300F0B3FB002821D00A20BE
:10715000FFF7D4FA04000B20FFF7D0FA164B050016
:107160001E78731E9E413B68F6B2191DD878FFF752
:1071700057FB3B682900DA7A043303929A7901932A
:107180000292009033002000059A04F0F5FD07B04C
:10719000F0BDFFF7B5FF002805D00620FFF7AEFAD7
:1071A00004000720D8E70820FFF7A8FA0400092008
:1071B000D2E7C046E064FF1FDC64FF1F70B50A4ED3
:1071C000040033780D00FF2B0DD0042004F05CFC8C
:1071D000011E08D0D0230370CE3B45708370C4706D
:1071E000307804F009FB70BD7443FF1F70B50400D4
:1071F00006200D0004F048FC011E0AD0D0230370C5
:10720000CD3B8370054B44701B688580187804F073
:10721000F3FA002C01D0FFF767FF70BDE064FF1F99
:10722000F8B5264F06003B680D001124002B05D150
:107230000522234B1B78134202D112242000F8BDF3
:10724000204A10241268002AF8D01278002AF5D0BB
:10725000DB0719D52B789A1E012A1AD80C2004F0C6
:1072600093FC132438600028E8D000230A224370DE
:1072700029000670023004F0E7FAFFF75BFF041EF6
:107280000AD0FFF731FFD9E700F012FB0028E1D167
:10729000E4E7002BE2D0D0E70B4B1B78032BCDD1DA
:1072A0001D20FFF72BFA094B18800028C6D0084B89
:1072B00004211878074A04F077FCBFE7E064FF1F59
:1072C000DD64FF1FFC64FF1FDC64FF1FDA64FF1F27
:1072D0000865FF1F60EA0000F7B50193194B140021
:1072E0001A78052306000F0012201A4221D0012926
:1072F00020D1154B1D68002D1BD002201F2C18D843
:10730000002C02D0019B002B13D0104B1F221E70AB
:107310006E1C0021300004F0FFFC019922003000B7
:1073200004F092FA310020002C70002F06D004F0F7
:1073300013FDFEBD064B12201D68DCE704F00CFBBC
:10734000F7E7C046DD64FF1FFC64FF1F7443FF1FA7
:10735000F864FF1FF8B50F4E12243368002B17D0C6
:107360001B780F3C834213D100250B4F0221387844
:1073700004F0C2FB094B042138781D8004F0BCFBEB
:10738000074B28001D8033685C7004F03DFA040050
:107390002000F8BDE064FF1F0865FF1FF464FF1FB5
:1073A000DA64FF1F70B5012823D11B4C2388002B02
:1073B00003D01A4A1578002D07D0194B1B68002BF3
:1073C00002D01878FFF7C6FF70BD3B2B02D93C3BBB
:1073D0002380F9E7134E0221307804F08DFBFA2266
:1073E0002388920002215A43307804F0ADFA2580B8
:1073F000EAE70B4B1B68002BE6D00B4B1B785B07B7
:10740000E2D5084B0221187804F076FB0022024BEB
:107410001A80FFF769FED7E7F464FF1FD864FF1FE7
:10742000E064FF1F0865FF1FDD64FF1FF8B51E4DF8
:107430002868002803D004F037FC00232B601B4E83
:107440003068002803D004F02FFC00233360184F6D
:1074500005243B7818002040234221D0154800F035
:107460002BFA3B78234213D0202004F08DFB2860B8
:10747000002813D02022002104F04EFC202004F02C
:1074800083FB041E306005D02022002104F044FC60
:10749000002004E0286804F007FC2C601320F8BDED
:1074A00000F00AFAF4E7C046FC64FF1FF864FF1F0F
:1074B000DD64FF1F6843FF1F10B50A4C23681A1EC6
:1074C0000ED0002808D10130587004F09DF9002832
:1074D00005D02368002B02D00021FFF787FE012290
:1074E000100010BDE064FF1FF7B5274E050033689C
:1074F0000191181E21D05C78244F012C30D1FFF768
:10750000FFFD002825D02000FFF7F8F804004128EF
:1075100014D91F4B022118781E4A04F045FB1E4B5C
:107520003C3C1C80022233685A703B78002B14D1FB
:1075300028000199FFF75AFE0120FEBDFA229200B1
:107540004243002AEED0124B0221187804F0FCF9D5
:10755000E8E7FFF7D3F80200F3E700233B70EBE71F
:107560003B78002BE8D1032004F08EFA011E08D0EE
:10757000D0230370CC3B457083703368187804F0D7
:107580003BF9FFF7B1FDD7E7E064FF1FD864FF1FA9
:107590000865FF1F60EA0000F464FF1F10B517497B
:1075A000838802008B4220D011D815498B4217D016
:1075B000144900205B1899B2012907D89268117804
:1075C0005A425341D8B2FFF7F9FD012010BD0E4ACF
:1075D00000209B1807229BB29A424041C0B2F5E7B7
:1075E00083681878FFF768FFF0E7836899785A781E
:1075F000090218781143FFF777FFE7E70A20000038
:1076000006200000F8DFFFFFAFDFFFFF014B18701F
:107610007047C0467543FF1F10B5064C207001F03F
:1076200041FA207804F038FB0521207800F062FD53
:1076300010BDC0460865FF1F0BB273B50D00002BCF
:1076400000DBC4E0884B187804F0DEFA041E0ED08C
:107650000378912B0FD0A22B00D1A1E0834B187897
:10766000FF2852D0210004F0C7F800284DD1802017
:107670000002684076BD43780F2B76D013D8052BD7
:1076800070D00E2BEAD18088794B98422BD8794B59
:1076900098421BD8784B9842E0D1A3681878591CBF
:1076A000FFF774F838E03E2BD8D18378032B74D0E1
:1076B0006CD8012B6ED0022BD0D1704B1B68002BE5
:1076C00023D05B68002B20D098471EE06C4BC0187D
:1076D0000C28C3D804F068FB1DC2C2150BC20B0BEB
:1076E0000B3223C23C00674BC0180728B6D8664B44
:1076F0001B68002B09D01B68002B06D02000984780
:107700000AE0A3681878FFF7C7F8200004F034FAFD
:10771000ADE7A068FFF762F800289FD0F5E7A368FF
:107720001B78002BF1D0554B1B68002BEDD01B684C
:10773000002BEAD0210055489847EDE74F4B1B68D6
:10774000002BE2D01B68002BDFD021005048F3E76C
:10775000504B1B68002BD8D05B68002BD5D0210084
:107760004348E9E7FFF7EAF9CFE780884A4B9842B8
:1077700003D04A4B984200D070E7464B1B68002B61
:10778000C3D05B68002BC0D02100D5E7153B012B8F
:10779000BBD963E7FFF798FAB7E7FFF77DFAB4E7DD
:1077A0003F4B1B78042B07D100236A4613800179D5
:1077B000408800F0C5FCA8E7364B1B68002BA4D01E
:1077C0005B68002BA1D00100364898479DE7012453
:1077D00021420AD0294B1B68002B04D05B68002B88
:1077E00001D000209847012043E78B070AD5264B9C
:1077F0001B68002B04D05B68002B01D02000984749
:10780000022036E70421280008400D4200D131E76C
:10781000254E3388002B21D0013B9BB23380002BB7
:107820001AD1FFF7DBF800280AD0204B1C70164B4A
:107830001B68002B04D05B68002B01D02000984708
:10784000FFF7C6F8694601F001FD6846FEF7FEFF46
:107850001D20FEF753FF308004200AE7024B187802
:1078600004F04AF9F8E7C0460865FF1F7543FF1F9B
:107870000E20000001200000091000000065FF1F1D
:10788000FEDFFFFFAFDFFFFF0465FF1F0C200000DE
:107890000B200000E864FF1F0D20000013200000F3
:1078A000DD64FF1FFFFF0000DA64FF1FD864FF1FC5
:1078B00010B501F09BF910BD014B18607047C04630
:1078C0000465FF1F0B880020162B01D81723042006
:1078D000014A13807047C046B264FF1F0020704702
:1078E000074A03001188814207D0918800209942FD
:1078F00002D101308000101870470020FAE7C0461E
:107900001065FF1FF0B58F7806000D00C5B01E2F63
:1079100015D1FFF7E5FF051E03D10024200045B077
:10792000F0BD00223B003100C078009200F0B2FBB5
:107930000400A81C00F0D2FBFF23EB70EEE7264BFF
:10794000062403931B78FF2BE8D0182FE6D87B087A
:10795000224A013BDB0002929A589446002ADDD06D
:10796000029AD3185B68002BD8D00878002802D17F
:107970004B78012B02D10624122FCFD107AFAB8851
:10798000697800976446AA68A047041EC6D1AB7800
:10799000029A5B08013BDB00D318390030005B68BA
:1079A0009847041E0BD1AB78042BB6D0039A310054
:1079B00010782200009700F06DFB0400AEE76A78B3
:1079C000002AABD1AA7805A93B88087130000A705B
:1079D0004B80FEF747FBA0E77843FF1FBCBF0011B9
:1079E0001D4B37B5050098420BD000290AD1FFF78F
:1079F00077FF002805D11948FFF772FF002800D053
:107A0000058037BD01291AD1FFF76AFF041EF8D09F
:107A100001235B420380A378FF2BF2D0FE2B07D01B
:107A20000023E0781422009329001E3300F032FB7B
:107A3000A01C00F053FB01235B426380E1E70229B5
:107A4000DFD1013901F0BEF80028DAD12800FFF7B4
:107A500047FF041EDFD1D4E7FEFF0000FFFF000058
:107A6000022210B5074B52421A80074801325A8051
:107A70009A80DA8000F07EFA044801F025F80020B0
:107A800010BDC0461065FF1F05790011E179001196
:107A90000388F7B50400002B02D102252800FEBDA3
:107AA00042680221137825485268FEF7A5FD002898
:107AB0002ED0234F01253A88002AEFD08023218839
:107AC0005B0201259B1A9942E8DC0C2004F05CF86B
:107AD000061E31D03B8822889C4600231800019561
:107AE00061469DB2491989B2AA421BD8002801D02B
:107AF00062443A8000233000082208C0210003F0CD
:107B0000A3FE104A1368002B13D100251660C5E7A9
:107B10006268022113780C485268FEF76DFD002858
:107B2000C7D1BAE760681D0140194181013301984E
:107B3000D6E71A001B68E6E71325AFE72AC0001155
:107B40007643FF1F0C65FF1F28C00011014B187002
:107B50007047C0467843FF1F14230A0010B51A402F
:107B6000194204D00122102101F048F810BD4B0643
:107B7000F9D4012088434000F8E710B514008B06C3
:107B800004D50122102101F039F810BD08230A00A4
:107B90001A40194202D14BB2002B0FDA102101F02A
:107BA0002DF8002808D02300F2331B78002BECD0EE
:107BB000F1342378012BE8D10020E6E70320890780
:107BC000FAD4E2E7F0B51F00184B85B01C680190AD
:107BD00002910392002C27D1200005B0F0BDA568CA
:107BE0003301ED186B89019A934211D3029A9342A3
:107BF0000ED8002F04D10A9B002B10D12C00EBE7EC
:107C00003B002978039A6868FEF7F6FC0028F2D159
:107C10000136B6B2A388B342E1D82468DAE7A36894
:107C20000A9A5B891380E9E70026F3E70C65FF1FDA
:107C300037B50C000A8849880123914217D3002ADE
:107C400015D0651D23792A0002210A48FEF7D4FCCD
:107C5000102300280BD023796188208800242A0073
:107C60000094FFF7AFFF0A23A04200D023001800C2
:107C70003EBDC0462AC0001113B50A0008884988D5
:107C8000012388420BD8002809D00024137905323B
:107C90000094FFF797FF0A23A04200D023001800AA
:107CA00016BD13B50A0008884988012388420BD8FD
:107CB000002809D00024137905320094FFF782FFD1
:107CC0000A23A04200D02300180016BDF0B58BB0E7
:107CD00003904A8808880E000123824255D3002869
:107CE00053D00023012704AC2370002271881300B5
:107CF0000092FFF767FF051E3ED02078002835D19F
:107D00002B78022B18D167706A8983000130E31841
:107D100080005A8069680222201803F095FD2378BC
:107D20000133DBB22370042B19D93B006889013081
:107D300080B2002BD9D01FE0022363701223584376
:107D40006A89231804305A8069681022201803F0C9
:107D50007BFD23780133DBB22370002BE5D10C4A85
:107D60006B899B185A425341DBB2DFE76378012BE2
:107D7000E4D12B78022BC7D022780A23002A04D022
:107D800021000398FEF798F9002318000BB0F0BD0E
:107D90000100FFFF0F4BF0B504001868002816D053
:107DA00083685D89A54207D88288AE18B44203DA99
:107DB00012019A18934201D10068EFE71E005F8913
:107DC0001036A74204D1002900D00D801800F0BD64
:107DD0003300EFE70C65FF1F70B505000C00088845
:107DE0000021FFF7D7FF03000120002B04D0220061
:107DF0002800197AFFF7C1FE70BDF7B50C00002509
:107E000001902300EE331B78AB4201D800200AE03A
:107E10006B00E65A00213000E718FFF7BBFF00288F
:107E200002D126800130FEBD017A0198FFF794FE51
:107E3000002802D03B882380F5E70135EDB2E0E76A
:107E400010B5040008880021FFF7A4FF03000120FB
:107E5000002B03D02000197AFFF77EFE10BD000032
:107E6000054B1B68002B01D1180004E09A68528969
:107E70008242F6D1988870470C65FF1FF0B50E2737
:107E8000002687B0039302ABFF183E8005001F4B0E
:107E900040891400984207D02B78013000976A6817
:107EA00080B2FFF78FFE060002212B7818486A681F
:107EB000FEF7A2FB00280FD06C892000FFF7D0FF4F
:107EC000002802D0013C0419A4B2039B002B00D06F
:107ED0001C80300007B0F0BD02212B780D486A6885
:107EE000FEF78AFB0028E7D102212B780A486A684E
:107EF000FEF782FB002807D0002EDED03B88A3428D
:107F0000DBD17489013CDFE76C89DEE7FFFF00000D
:107F10002AC0001128C0001126C0001110B50C00A5
:107F2000FFF7DEFC03000220002B0AD0002C00D05B
:107F300023609B781720FE2B03D00138FF2B00D144
:107F4000002010BD73B50D0001A904001600FFF755
:107F5000E5FF172805D0002E04D129002000FEF7E8
:107F600027F976BD01221021200000F047FE0028ED
:107F7000F3D0F6E7014B18607047C0461C65FF1F41
:107F800037B56B469D1D010004000222280003F056
:107F90008BFD2B88B02B0ED12379122B09D1230016
:107FA000FA331B78012B06D10121608800F0E0F83C
:107FB00001E01B2BF8D037BD10B5054B042118701C
:107FC00000F098F8FFF74CFDFEF770FB10BDC046BF
:107FD0002065FF1F0020F0B50BB20F0087B0834271
:107FE00034DA274B187803F00FFE051E2BD00378E8
:107FF000A02B25D103AE3100FEF7E4F8041E0BD10F
:10800000B378DB0724D51F4B06341B68002B03D045
:108010003100688898470400A868002801D003F060
:10802000F3FC002C08D1184A039B1340174A9342D3
:1080300006D0B3781B2B03D00121688800F098F894
:10804000280003F099FD80200002784007B0F0BDC1
:108050000F4B1B68002B10D0310068889847041E16
:10806000DAD07378002BD7D1B27801A90A704B808F
:108070000C716888FDF7F6FFCEE70624F1E7C046ED
:108080002065FF1F1865FF1F00FFFF0000011200A1
:108090001C65FF1FF7B50190FC200D0017001E00A6
:1080A00003F0F2FC04001320002C12D0B0232000B7
:1080B0002370089BF4226770658026710830002BBE
:1080C00008D0190003F0C0FB2100019803F094FBD5
:1080D0000020FEBD089903F01FFEF5E710B5041E51
:1080E00006D00078FD2803D803F0A6FCFF232370F8
:1080F00010BD00000A1F93B210B504000220032B2C
:1081000005D882400020024BD1529B189C7010BDB4
:108110004065FF1F0B8870B5043B04000D00022072
:10812000032B0BD80121200000F04CFD030014208C
:10813000002B03D02900200000F0DEFB70BD000002
:1081400007B51300034A00920A00012100F02CFC3D
:108150000EBDC0467D83001107B501920322009237
:10816000024B0A00122100F049FC0EBDFB830011F6
:1081700007B56B4601AA11800449D88008780633F8
:10818000012802D1190003F01FFB07BD2165FF1F65
:108190000C4B10B518700023FF210B4A138013817C
:1081A00093819380094A5380137051729381937223
:1081B000D174D3821375517703F04EFB00F0FCF9B4
:1081C00010BDC0465065FF1F4065FF1F2265FF1FA1
:1081D000F0B58DB06B46002003910C229B5E83426C
:1081E00000DBB0E05D4B187803F00EFD051E00D1FA
:1081F000A4E00378902B00D09DE006AF01004688F4
:10820000380000F013FA79680400002900D19CE0DE
:108210003B88052B6ED13B89032B1CD905AC200074
:1082200000F0A2F86288172A61D83989131D994293
:1082300031D17968237804310291D90738D5607833
:1082400000F08EF9071E06D0002303712378012B5E
:1082500008D0132B23D0A868002800D178E003F0C1
:10826000D3FB75E06288029909A800F0A6F8029095
:10827000380000F08BF909AA2378387A019200229D
:1082800031000092029A00F012F9380000F064F90F
:10829000029B002BDFD0300000F080F9DBE7037891
:1082A000032BD8D16288029909A800F0D6F8DEE73E
:1082B000122B13D1029909A800F0B5F8021EEAD1D9
:1082C00027498B88002BC6D0887909A9237801918A
:1082D00061780091310000F0EAF8BCE7002302AABF
:1082E00093833000617809AAFFF72AFFB3E71D4B9B
:1082F0000993F6E7042B02D09A1F012AABD8184A3B
:10830000043B9B00995A0029A5D0D21890783100DF
:108310003A0000F0AEF800289DD13B88042B03D032
:1083200001213000FFF724FF012C04D1A8680028A8
:1083300001D003F069FB280003F01EFC8020039BA2
:108340000002434018000DB0F0BD012800D182E7C3
:1083500001213000FFF70CFFEDE7C0465065FF1F1D
:108360004065FF1F010017000B7803704B784370C6
:10837000CB788A781B021343438070470A88030036
:1083800002700A88120A42700A88012A06D14A88B5
:1083900082704A88120AC27004207047022082420A
:1083A000FBD14A8804309A704A88120ADA708A88A7
:1083B0001A718A88120A5A71EFE710B50400012079
:1083C00082420CD94B780A781B02134323808342E4
:1083D00006D1CB788A781B0213436380002010BD3E
:1083E000022BFBD1CB788A781B02134363804B7935
:1083F0000A791B021343A380F0E70B8803700B88F4
:108400001B0A43704B8883704B881B0AC3708B8890
:1084100003718B881B0A4371CB888371CB881B0A3D
:10842000C3710820704703000120082A14D14A783C
:108430000878120202431A80CA788878120202432E
:108440005A804A790879120202439A80CA79887957
:10845000120202430020DA80704710B504000120A8
:10846000022A05D100204B780A781B02134323808F
:1084700010BDF8B5060010200F00150003F004FB36
:1084800004000120002C0ED0A0230C222900238000
:108490006780201D002D07D003F0D6F921003000A1
:1084A00003F0AAF90020F8BD03F036FCF6E7F7B5B3
:1084B0001E00009008AB142017001D78019103F0F6
:1084C000E3FA041E12D0A2230370019B477043807D
:1084D000099B057146710C220830002B07D019004A
:1084E00003F0B2F92100009803F086F9F7BD09996D
:1084F00003F012FCF6E737B5041E0FD04388002BBB
:108500000CD00025C1881323007A1722019500950D
:10851000FFF7CDFFFF2365806372257037BD000034
:1085200010B50C4904004A88002A09D08B89002B19
:1085300005D00020CB8A0222834201D010BD012247
:1085400013000A20434300204032C854C818428018
:108550000472F3E72265FF1F002343800370704716
:10856000094B00211A0010B55C88002C06D01C793C
:10857000844203D10A234B43D01810BD01310A3382
:108580000329F1D10020F8E72265FF1F10B5040090
:10859000407A03F051FAFF23637210BD7047043034
:1085A00010B580B203F058FB002803D004214942E3
:1085B00003F08AFA10BD000070B50025104CA068C9
:1085C0002580A581A580A84202D003F01DFAA560F0
:1085D00000250C4C0C4B606D1D80230058331D7022
:1085E000A84202D003F010FA6565002560680028F3
:1085F00001D003F009FA013508340A2DF6D170BD17
:10860000E865FF1F8C65FF1FDC65FF1F70B5041E4A
:1086100009D1054D2880A881A880A868002802D02B
:1086200003F0F2F9AC6070BDE865FF1FF0B54B8850
:1086300085B00193002343600A7905000F00022AE8
:1086400000D07BE0CA88032A17D98B685E78197836
:108650003602DC78D8790E4399781B7A24021B0203
:108660000C43034353495BBA0B80331D93421ED125
:10867000042C04D0631F022B0ED9012015E0019AAF
:108680004D4B1201D35A002B06D00198FFF7BEFFC5
:108690004A4A1369013313610421B8682E812C8082
:1086A000494203F011FA6860002005B0F0BD434D67
:1086B000042C06D0631F022B0FD9EB680133EB604B
:1086C000DBE7019A3C4B1201D35A002B05D00198ED
:1086D000FFF79CFF2B6901332B61374B300002936E
:1086E000019B029A1B010193002301998C468B5236
:1086F000130063449C8003939E81FFF750FF039B0C
:10870000041E986016D00421B868494203F0DCF9D1
:10871000FA880100043A200003F096F80199029AC1
:10872000FB888A5A043B9B18029A8B522B680133B0
:108730002B60A2E7AB690133AB619EE71E4B02934E
:10874000019B1E01029BF35A002B2DD002998C191C
:10875000A068002828D0012A26D1FA889B189BB24D
:108760007352A189994217D39B1AC018B96803F0B4
:108770006BF8029BA289F35A934200D07DE7002256
:108780002B81A3882B80A3686B60029BF2520B4A5B
:1087900053680133536070E7084A9368013393606C
:1087A0000198FFF733FF68E7044A536901335361C7
:1087B000F6E7C0465265FF1FE865FF1F5865FF1FBB
:1087C00070B5051E15D10B4C0B4B18802300583388
:1087D0001870606D002802D003F016F96565250059
:1087E00050356068002801D003F00EF90834AC421F
:1087F000F7D170BD8C65FF1FDC65FF1FF0B517005A
:10880000A12285B0920001934243394B06001B68B8
:108810000C009B18D933FF331D78FDF741FF04305E
:10882000854204DD3000FDF73BFF0430C5B2BD4298
:1088300007D33A0000213000019B03F09DF805B0FA
:10884000F0BD2900380003F09FFA2300C6B2503370
:108850001E700393019B29006365380003F06CF9D7
:10886000CBB20293002B02D0039B01361E70002670
:108870002300503303931B78B34204D8606D002863
:1088800031D10020DBE7029A2800002A04D0013B06
:108890001000B34200D02800F700E719387003F049
:1088A0002BFA786000280ED03A78019902F0CCFFBC
:1088B000019A3B780136D3180E4A0193D369F6B278
:1088C0000133D361D4E7039B18706065A74205D1DB
:1088D000084A1320D36A0133D362B0E7606803F01B
:1088E00093F80834F2E703F08FF800236365C8E7D4
:1088F0003409FF1F5865FF1FF7B50D00070004215D
:10890000686803F0E1F82B89040003702B891B0AC7
:1089100043702B8883702B881B0AC3702E89022515
:108920000436F6B2F42E15D81B4B9F4214D10C20FE
:1089300003F0AAF81135011E0CD0902303708E3B72
:108940000371043B4380154B8460C680187802F0A5
:1089500053FF00252800FEBD5C237B43104AD3183B
:108960000093583301931B78002B0FD10300320082
:1089700038000099FFF742FF019B05001B78002B90
:10898000E8D13800009902F027FFE3E7054A072500
:10899000536A01335362DDE7FEFF00005065FF1F9D
:1089A0008C65FF1F5865FF1FF0B587B0009017203A
:1089B0000F0016000193FFF7F2FD1325041E19D0D6
:1089C0000C98031E02D00199201D9847030AE370FA
:1089D000052302AAA0700430908127700098667069
:1089E00003A993800494FFF787FF051E02D020009F
:1089F00003F00AF8280007B0F0BD0000F0B587B01A
:108A00001F000CAB1B780391059301210DAB0600F1
:108A10001C78049200F0D6F81425002821D02000FC
:108A2000FFF77EFD0135041E1BD01149059B0A7816
:108A300003700132D2B2131EC68001D101231A0085
:108A40000B7022713000049B03990097FFF7ACFF75
:108A5000051E09D1230021000648074A093303F007
:108A6000ABF9280007B0F0BD002363802370F8E75E
:108A70005465FF1FF784001130750000F8B505003C
:108A80000E00064C064F2368002B02D03100280050
:108A900098470434BC42F6D1F8BDC046F865FF1FC4
:108AA0000C66FF1F0123064A5B42538000231371AB
:108AB0005362044A136053609360D360136170473C
:108AC0000C66FF1FF865FF1F0200002310B5064962
:108AD0009C000859002801D1625010BD0133052BBC
:108AE000F6D11320F9E7C046F865FF1F034A538803
:108AF000181A434258414042104070470C66FF1F0D
:108B0000F0B585B002930AAB1F780CAB1B880090C0
:108B100008000E0001920393FFF7E8FF0500112003
:108B2000002D1BD10E48FFF7E1FF04001520002C9B
:108B300014D006220B99A771E01D02F085FE019B5F
:108B400030002371029B29006371009B66802370B3
:108B5000039B6562E381FFF791FF280005B0F0BD3C
:108B6000FFFF000010B5FFF7C1FF04000220002C3A
:108B700012D060880121FFF781FF606A002801D0D0
:108B800003F092F828220021200003F0C5F8012309
:108B900000205B426380207110BD000030B5074AA1
:108BA000074C5588010013780020A54204D05B1AB9
:108BB00059424B415842104030BDC0460C66FF1F21
:108BC000FFFF0000084A10B501230C00904208D0B6
:108BD000FFF78CFF031E04D0037923405A1E9341F4
:108BE000DBB2180010BDC046FEFF0000024B187932
:108BF000431E9841C0B270470C66FF1F70B5040059
:108C00000D001600FFF772FF002804D10D4B9C42A7
:108C100000D0143070BD416A03790520002907D0C7
:108C200012221A40102A02D10520002EF2D10F2064
:108C3000DB06EFD5897E0C20A94289414942494291
:108C40000840E7E7FEFF0000030010B5002800D150
:108C500010BD0348034A41889142F9D09847F7E78D
:108C60000C66FF1FFFFF0000002330B5C45CCD5C25
:108C70006C40D4540133102BF8D130BD0F230022A7
:108C800010B5C45C64002243CA54C25CD209013BE3
:108C9000F7D210BD0200010010B52032103102F0F1
:108CA00033FF10BDF0B58BB0039010200593170073
:108CB000049102F069FF0090102002F065FF009B14
:108CC00013240190002B05D000280CD11324009808
:108CD00002F0EAFF019B002B02D0180002F0E4FF33
:108CE00020000BB0F0BD102002F04EFF0600102057
:108CF00002F04AFF13240500002E00D1AEE0002848
:108D000019D01022002103F007F83200290003983F
:108D100002F0FAFE041E0ED133787F2B51D83000BA
:108D20000099FFF7ABFF009B1B787F2B53D801996D
:108D30000098FFF7A3FF300002F0B6FF002D02D02D
:108D4000280002F0B1FF002CC1D1102002F01CFF5E
:108D50000600102002F018FF0290002E7CD00028A0
:108D600078D03A000F3223000125121105D00F33BD
:108D70003B4015B25A4253411BB26A1E1201002BEE
:108D800033D0049BD2B298180099029AFFF76CFF77
:108D9000013D10220021300002F0BEFFADB2049F61
:108DA0002D017D19AF4242D0002C33D0300002F0AB
:108DB0007BFF029B002B00D189E7180002F074FFB3
:108DC00085E729003000FFF759FF28002549009A60
:108DD000FFF74AFFA7E729000098FFF74FFF280099
:108DE0002049019AFFF740FFA5E70F210F400499A2
:108DF0008A18D9B28F4208D9D15C06A81954013318
:108E0000102BF6D1029A0199C0E7791A48424141E4
:108E1000C901F2E73900300006AAFFF725FF32004A
:108E2000039806A902F070FE10370400BAE7002C80
:108E3000BCD13000029906AAFFF716FF320006A93E
:108E4000039802F061FE082204003100059802F048
:108E5000FBFCABE71324A9E71324AAE7002800D002
:108E60006EE733E730C00011F0B58BB00F0016008D
:108E70000225009000283FD0002A3DD00B1DDBB218
:108E80001800029302F080FE1135041E34D0FDF765
:108E900047FD05003A000099201D02F095FEEBB257
:108EA0000393E3702B0CDBB22F0A00936370FFB2C5
:108EB0002B0E2370A7700193FDF72CFD10220100EB
:108EC00006A802F081FE2100029A04AB06A8FFF773
:108ED000E9FE051E0DD1039B08223370009B04A9F7
:108EE000B370019B7770F370301D02F06DFEFDF7DB
:108EF0001DFD200002F0D8FE28000BB0F0BDF0B53B
:108F00008FB00D00149E039004920593002A03D1A4
:108F1000022420000FB0F0BD002EF9D00398FFF717
:108F2000E5FD1424071EF4D07278337812021A4338
:108F3000B3781B041343F27812061A43036A0192B2
:108F4000934201D30133E3D1002D03D03B790124B7
:108F50009B07DED50822002106A802F0DDFE059B56
:108F600013240433DBB21800029302F00DFE051E39
:108F7000CFD0059A0499043002F026FE0422310075
:108F8000280002F021FE3900102210310AA802F058
:108F90001BFE2900029A06AB0AA8FFF783FE041EF7
:108FA0000FD1082206A908A802F00EFE0822311DE2
:108FB00008A802F071FC012807D101990398FDF778
:108FC000C9FC280002F070FEA3E70124F9E70000C5
:108FD00070B51C4C05002368181E10D0002D14D14C
:108FE0001A78002A0CD1981C083202F02DFC02F0ED
:108FF0001BFC0135002808D123681D70012070BDBD
:109000000A331800082202F01FFC2368002BF5D059
:10901000122002F039FD061E0DD0C1232168037015
:10902000457002311022023002F00EFC236831003C
:10903000587802F0E1FB206802F036FE002323603E
:10904000DCE7C0463466FF1FF8B504002020FDF7BA
:1090500055FB0D4EA700BB590500002B0DD0002875
:109060000BD0D878FF2809D108492A000C55F359AC
:1090700007480333611802F09FFEF8BD290002F093
:1090800013FC0028F0D1F8E75066FF1F3866FF1F79
:10909000A1A2001170B5064D84006359002B05D0C4
:1090A000D87802F0C9FCFF226359DA7070BDC0465F
:1090B0005066FF1F70B506008CB00C001500002133
:1090C0003022684602F028FE31001022684602F085
:1090D0007BFD1D2021000322684402F075FD6846D7
:1090E000FFF7D8FD2D21040003222800694402F077
:1090F0006BFD20000CB070BDF0B50700160097B0F6
:1091000001931CAB1D7830221EAB00910AA80021F0
:109110001C7802F001FE102239000AA802F054FD6A
:109120001022002102A802F0F7FD0722310002A858
:1091300002F04AFD072202AB9818631E9C41019978
:1091400002F042FD02AB9C732B005A1E934102AA0F
:10915000D3730021102206A802F0DEFD06221D991D
:1091600007A802F031FD1A2002ABC01806221F9991
:1091700002F02AFD102200990EA802F025FD10220F
:1091800002AB0EA908781C78013A6040D2B2087090
:1091900001330131002AF5D10AA8FFF77BFD102227
:1091A00012A904000EA802F04FFB102206AB0EA974
:1091B00008781D78013A6840D2B208700133013155
:1091C000002AF5D10AA8FFF765FD04431022209874
:1091D000E4B212A902F0F8FC200017B0F0BD70B59F
:1091E0000E0014008CB00100102268461D0002F031
:1091F000EBFC3100082204A802F0E6FC2100082262
:1092000006A802F0E1FC6846FFF744FD04001022C6
:10921000280008A902F0D8FC20000CB070BDF8B5F9
:1092200006000D0000243719AC4200D3F8BD02F04F
:10923000B3FA030A3B70631CDBB201379D4203D9CA
:109240000234F054E4B2EEE71C00EDE773B506001B
:109250000C000225002819D0002917D0032101A8ED
:10926000FFF7DDFF6B469A793F231A400133134322
:109270006A463000937101A92200FFF71BFF051E0B
:1092800004D10322E01C01A902F0DEFA280076BD19
:1092900003785807DA08C00FD20080009B071043FC
:1092A0009B0F1843C0B2704707230B40C908C90081
:1092B0000B4303707047000070B50400FFF7EAFE2F
:1092C000134DA4006359002B21D0186A002801D047
:1092D00002F0EAFC2B59986E002801D002F0E4FC61
:1092E0002B59D86E002801D002F0DEFC2B59186FE4
:1092F000002801D002F0D8FC2B59586F002801D06B
:1093000002F0D2FC285902F0CFFC00232B5170BD93
:109310005066FF1F0E4B8000C35870B50C00002B29
:109320000FD09D68002D0CD02B78201D0B706B7812
:109330004B70A97CFFF7B8FF2B7E23726B69E3604B
:1093400070BD10220021200002F0E6FCF8E7C046C4
:109350005066FF1F014B18607047C0464C66FF1FE8
:10936000074A03008000825810B5002A06D0D08832
:10937000984203D1012901D1FFF79EFF10BDC046DD
:109380005066FF1FF0B5264E95B087000B93BB5972
:109390000500099112200A92002B31D0D888FFF7DE
:1093A000A5FB04001420002C2AD0280010A9FFF7E8
:1093B000B1FFBB591E781D6A002E23D00895FDF71A
:1093C000EFFA07000020FDF7F1FA0790A379E61DF8
:1093D000069310AD0CA9089800F0E2FA0EA9280037
:1093E00000F0D7FA0B9B0A990493069B0998029305
:1093F000079B0396019300970EAB0CAAFFF77CFE28
:1094000015B0F0BDFDF7CCFA06903000FDF7CEFAAE
:10941000E31DA779079310AB06000893DAE7C0466F
:109420005066FF1F30B50C4C85002A59030085B0EB
:109430000120002A0ED018006946FFF76BFF2B5958
:109440001A78D888054B002A00D1054B6A460721B7
:1094500000F0D9FB05B030BD5066FF1F9399001195
:10946000A199001130B5094C8500295985B0102209
:109470006846253102F0E8F92A591121044BD088B9
:109480006A4600F0C0FB05B030BDC0465066FF1F05
:109490003D9A001130B5094C8500295985B010223C
:1094A0006846353102F0D0F92A591121044BD08891
:1094B0006A4600F0A8FB05B030BDC0465066FF1FED
:1094C0007B9A0011F7B54D4F86001020F4590D001E
:1094D00002F05AFBF3592062186A132200286CD05C
:1094E000033A29009C6802F0AFF9F3591A78019207
:1094F000002A58D11E6A227D317B944651400122B8
:10950000019F114201D167461740217D91433943A4
:109510002175377B4F40BC4660460027800701D449
:109520004F081740012102208F40227D82433A4399
:109530002275377B5740BC4660460027400701D460
:1095400097080F400420227DBF0082433A432275D2
:10955000627D002794466046727B42400A4201D1F8
:1095600067460F400121627D8A433A436275777BEB
:109570005740BC4660460027800701D457080F407B
:109580000220627D7F00824317436775767B00224D
:109590007E40760701D4BA080A400426617D920015
:1095A000B1430A4362756A78002A08D06278002ABB
:1095B00005D005220533DA7700221000FEBD042213
:1095C0002979114205D1A17C114202D10533033A18
:1095D000F1E7019A21782C78002A02D10A002100B3
:1095E000140018220429E8D8042CE6D8052060438A
:1095F000034A05331218525CDDE7C0465066FF1F70
:1096000040C0001110B50A001121024B00F0FBFA16
:1096100010BDC046D79A00110B0030B587B001AD20
:109620002B806B4604001100981D082202F00CF9F3
:109630002A000B212000024B00F0E5FA07B030BDF4
:10964000FF9A001110B50A001121024B00F0DBFA5D
:1096500010BDC046539B001113B50B0011006A46A4
:1096600013706B4604000622581C02F0EDF86A469F
:1096700008212000014B00F0C6FA13BD739B0011B6
:1096800010B50A001121024B00F0BDFA10BDC04612
:10969000C39B00117FB505000B4BAA00D4580800EE
:1096A000002C0FD0666F237FE28821780396266F07
:1096B0000296E66E0196A46E0094FDF709FC280060
:1096C000FFF7FAFD7FBDC0465066FF1F10B517219A
:1096D000FFF7E0FF10BD000070B50A000D00064B5B
:1096E0000221040000F08FFA060029782000FFF71D
:1096F000D1FF300070BDC046A39A001170B586B08E
:1097000000236A461370836804001D78681E0A28C7
:1097100059D801A902F048F9060633373B3F4347C1
:109720004B4F5300180000F042F9062312284BD08B
:1097300000281BD16088FFF7D9F90823002813D02F
:109740004279002A47D1264B1A78072312070BD5F6
:10975000244B1A680723002A06D01668002E03D06F
:10976000290001AAB04703006A4613706B461B78B4
:109770006088002B2AD1FFF767FC06B070BD180087
:1097800000F06CF9D4E7180000F087F9D0E7180072
:1097900000F093F9CCE7180000F0ADF9C8E7180025
:1097A00000F0C3F9C4E7180000F0F6F9C0E71800AC
:1097B00000F0F6F9BCE7180000F013FAB8E718005B
:1097C00000F013FAB4E707236A461370694660880D
:1097D000FFF782FFD1E70523012AC5D1024BB8E785
:1097E000DD64FF1F4866FF1F4C66FF1FF8B52C4F56
:1097F0008600F35904000D00002B40D0DA88824225
:109800003DD15A78062A33D11A78002A2ED0012069
:1098100099681A6A097D014206D0157B054203D07A
:1098200007225A700120F8BD0220014204D0157BA6
:10983000054201D00922F4E70420014204D0127B42
:10984000024201D00B22ECE7164B1B68002BE9D03B
:109850005B68002BE6D020009847BB5900215B785D
:10986000122BDFD12000FFF715FFDBE70E4BECE7F3
:10987000112A04D1002900D032252900F2E7002D59
:1098800008D12000FFF732F9002803D01023027915
:109890001343037121002800FDF798FAC2E7C04680
:1098A0005066FF1F4866FF1F4C66FF1F70B50E4EC7
:1098B0008500AB590400002B13D01B78002B11D16D
:1098C0000A4B1B68002B04D05B68002B01D02000E2
:1098D000984773595B78122B03D100212000FFF7C2
:1098E000D9FE70BD024BECE75066FF1F4C66FF1FB0
:1098F0004866FF1F094B8000C3581020002B0CD076
:109900001A6A002A09D09B68002B06D0127A1B7EA7
:10991000101C9A4200D9181CC0B270475066FF1F35
:1099200070B503000D0014000220002A30D0002979
:109930002ED013700B78081D53704B789370FFF77F
:10994000A7FCE070012002212B7A23716B7B03407E
:1099500063716A7B0A401343042263716E7B164075
:10996000334363716E7BF608F600334363712B7BE0
:109970000340A371287B014000200B43A371297B86
:109980000A401343A3712A7BD208D2001343A37168
:1099900070BD10B50A0001000120FFF7C1FF10BD26
:1099A00010B50A0001000220FFF7BAFF10BD70B524
:1099B00006000C000220002E30D000292ED0737833
:1099C000201D0B70B3784B70F178FFF76DFC01220E
:1099D0003579257271794B1008001340934010407F
:1099E0000343881010408000C9080343C9000B439B
:1099F0006373B1794B100800134093401040034348
:109A0000881002409200C9081343C9000B4321206B
:109A10002373FCF773FE854201D2122070BD222011
:109A2000257AFCF76BFE8542F7D823781820042BA3
:109A3000F4D86378012BF1D80020EFE7030010B5CC
:109A40000220002909D0002B07D00322481C0A70ED
:109A500019000D3201F0F8FE002010BD03000222B3
:109A6000080010B5002B06D0002904D00E32591C76
:109A700001F0EAFE0022100010BD030010B5022024
:109A8000002909D0002B07D00422481C0A701900B5
:109A90000C3201F0D9FE002010BD10B5FFF7DEFF3B
:109AA00010BD03000220002906D0002B04D005229F
:109AB00000200A701B784B70704703000220002BB7
:109AC00008D0002906D05B7800200B70013B082BE2
:109AD00000D918307047030010B50220002909D0C2
:109AE000002B07D00622481C0A7019000A3201F028
:109AF000ABFE002010BD10B5FFF7B0FF10BD020097
:109B00000B00022010B500290ED0002A0CD007212E
:109B10001970118859701188090A99701118082252
:109B2000D81C01F091FE002010BD03000A000220A5
:109B300010B5002B0CD000290AD09978587809026A
:109B400001431180901CD91C082201F07DFE0020E9
:109B500010BD030010B50220002909D0002B07D04A
:109B60000822481C0A701900921801F06DFE0020AE
:109B700010BD02000B00022010B500290BD0002AF6
:109B800009D009211970117818185970511C062232
:109B900001F05AFE002010BD10B5FFF75FFF10BDA9
:109BA00002000B00022010B5002A09D0002907D0BE
:109BB0005178197011180622581C01F045FE00203A
:109BC00010BD030010B50220002909D0002B07D0DA
:109BD0000A22481C0A701900063201F035FE0020E6
:109BE00010BD10B5FFF73AFF10BD02000B000220B8
:109BF00010B5002A06D0002904D018005178FFF7CC
:109C000053FB002010BDF0B585B017001E006A465A
:109C100006230500080091819380FEF7C0FC132401
:109C2000011E02900CD03800B047041E05D1280058
:109C300001A9FEF76FFA041E02D0029801F0E4FEBB
:109C40002800FFF701FA200005B0F0BDF0B50400D0
:109C50008BB0019115000021102202A802F05CF8DF
:109C6000334EA700B85900283CD0C388A34239D14D
:109C70000378002B36D14278062A18D10200010061
:109C8000553235310C3006ABFFF7A9FA002829D13F
:109C90002000FFF72FFE020006A902A801F0D4FD64
:109CA000200002A901F0F0FF01200BB0F0BD816E91
:109CB000002917D00B8A112A28D19D420ED1019874
:109CC0001231093A01F0E8FD012807D1BB59200003
:109CD0009D6EFFF70FFE29000200DEE73221200013
:109CE000FFF7D8FC2000FEF701FF061E1BD0416ADB
:109CF000002918D00B8AAB4215D1082201981231E5
:109D000001F0CAFD01280ED1716A0AE09D42E9D135
:109D100008220198123101F0BFFD0128E2D1BB59A0
:109D2000996E8A7EB9E7200001F0A6FFBCE7C04625
:109D30005066FF1FF0B56B4D87007E5985B03378B4
:109D400002900393002B00D087E0B368346A01933C
:109D50007078062817D101221B7D134202D0217B87
:109D6000114218D10222134202D0217B114251D15B
:109D70000422134203D0237B134200D08BE0019BCB
:109D80005A7DEB5991E007380428F8D801F00CFE11
:109D9000032E42678300B36E002B03D11C2001F019
:109DA000F3FEB066EB599C6E002C1CD010220021F3
:109DB000200001F0B1FF0298FFF79CFD0100200098
:109DC000FFF72DFA01F0E8FC208220000821123074
:109DD000FFF725FA0298FFF78DFDA076EB592100D9
:109DE000D888FFF70FFC0822EB591CE0B36E002B5C
:109DF00005D01A00198AF0881232FFF70DFC0222F2
:109E0000019B197DEB5911423DD0207B10423AD085
:109E1000073208E0F488FCF7DBFD01002000FFF7C3
:109E200011FC0A22EB595A70029B9C002A59537864
:109E3000073B042B11D8D088FEF758FE00284ED0DF
:109E4000C3895A08D2182849029B0298CB542B592F
:109E500041180433254801F0AFFF05B0F0BDFCF711
:109E60009FFD03000120834201D100200393EB59A1
:109E7000DE88FCF79BFD039902003000FFF7ECFB46
:109E8000019AEB59117D042211420CD0217B114221
:109E900009D00B22C7E7F688FCF73CFD0100300033
:109EA000FFF7EEFB6BE7019A527D01210A4204D0D5
:109EB000607B084201D00C22B5E702210A4204D09F
:109EC000607B084201D00E22ADE704210A4204D093
:109ED000627B0A4201D01022A5E71222A3E7FA22F0
:109EE0005200B0E75066FF1F5466FF1FABA200117F
:109EF00010B5064B1A780423100018401A4200D0FF
:109F00000348FFF727FA002010BDC046DD64FF1F9D
:109F10007C43FF1F70B50400FFF7D4FA051E43D140
:109F20002000FFF77FFA234EA400A0598268937C9B
:109F3000DB0708D50321036A1B790B40012B02D1F3
:109F4000017F0B430377431DD97F8B1E022B0DD856
:109F5000022900D00121C088FCF790FF0421335969
:109F60001A7F59700A431A77280070BD01290CD155
:109F700002231022437000210C3001F0CDFE305935
:109F800010213530FFF74BF9EEE70529ECD102231C
:109F9000D118437010220C3001F056FC04233259C2
:109FA000117F0B431377EAE708251828DCD1053D1C
:109FB000DAE7C0465066FF1FF0B58BB005914388C5
:109FC0007E4F9E00F45915000493002C15D10129F1
:109FD00002D000200BB0F0BD101D57781678FFF7A7
:109FE00057F9EB68320002932B7A049901930090A1
:109FF0003B002000FCF70CFFEBE7E388049A934258
:10A0000001D00820E6E72378012B00D1D4E0059B9E
:10A01000581E092800D9CFE001F0C6FC05CE0A2958
:10A02000CC506C859AB229000498FFF773FFD1E7F2
:10A03000200029001022453001F006FCB9594B7868
:10A04000042B02D1013B4B70C3E70B000A00253300
:10A0500035320C310498FFF795F90498FFF702FAAE
:10A060000522431E9841BB59C0005A70B2E7200038
:10A0700029001022553001F0E7FB049B4F4C9D0056
:10A08000295904980A0006AB55320C31FFF77AF9CA
:10A0900029591022453106A801F0FEFB012808D1FC
:10A0A0000498FFF7F7F90590002804D106222B59F0
:10A0B0005A7005988EE708230593FAE763780C2B0E
:10A0C0007AD1E36E002B03D11C2001F05DFDE06628
:10A0D000BB59D86E00286FD01022290001F0B4FBC4
:10A0E000BB590498DC6EFFF705FC0D22A076BB5926
:10A0F0005A706EE7E06E00285ED063780D2B5BD15E
:10A100002B8808220382A91C123001F09DFBBB5949
:10A110009A68517D0222114226D0186A407B104273
:10A1200022D00C32E4E763780E2B45D1236F002B4D
:10A1300003D1162001F028FD2067BB59186F0028B5
:10A1400003D01022290001F07FFB0F22BB59CFE77B
:10A1500063780F2B30D1206F0622691C103001F07C
:10A1600073FBBB599A68517D0422114203D0196ACE
:10A17000497B1142D5D100210498FFF78BFA28E7DB
:10A18000636F002B0DD0BB59586F0028F3D01022FD
:10A19000290001F059FB0122BB5952425B6F1A6141
:10A1A000E9E7142001F0F0FCBB5960675B6F002BFE
:10A1B000E9D126E72978DFE707200BE75066FF1F84
:10A1C00010B5064C207001F007FC06212078FDF741
:10A1D00091FF0348FEF778FC10BDC0466366FF1F81
:10A1E0006193001100200BB270B50D00834216DAA6
:10A1F000264B187801F008FD041E0DD00378922B31
:10A200000ED0A02B37D0224B1878FF283AD021004F
:10A2100001F0F2FA002835D180200002684070BDBC
:10A2200043780E2B0BD03E2BEDD18378052B12D02B
:10A23000082BE8D181798088FFF7D8FA08E0154B20
:10A2400082889A42DFD183681878591CFEF7C0FED5
:10A25000002817D1D7E7104B1B785B0712D50F4B9F
:10A260001B68002B0ED09B68002B0BD0C289811D70
:10A2700080889847ECE7FFF741FAA068002801D0F2
:10A2800001F0C2FB200001F077FCC5E76366FF1F09
:10A290007543FF1F18200000DD64FF1F4C66FF1F81
:10A2A00010B50078FFF712FA10BD10B50078FFF76F
:10A2B000FDFA10BD0C234343084A10B59B185A6899
:10A2C000002A03D0012901D1904710BD9B68002BC3
:10A2D000FBD00029F9D19847F7E7C0468066FF1FF9
:10A2E00001238340094A10B5946B1C439463506B5F
:10A2F00098435063D46B20009843012901D120007A
:10A300001843D063116B0B43136310BD00800040F2
:10A31000F0B500240127154B85B0DA6B144E03927B
:10A320001A6C0192DA64019BE3403B4217D0039D13
:10A33000E5403D400295E5B202992800FFF7BAFFDB
:10A34000316A736A002908D03900002B01D00299C4
:10A3500079402800FFF7C4FF01E0002BF9D1013458
:10A360000C36172CDFD105B0F0BDC0460080004090
:10A370006466FF1F064B01215A68C2400A4204D09E
:10A380001B68C3401800084070471B6DF9E7C046C2
:10A39000008000400122064B8240002903D0D9688A
:10A3A0000A43DA607047D9689143D960FAE7C0463A
:10A3B0000038004030B5032444430F4BE25C1B19C6
:10A3C0009C785D7801232D1B0135AB40013BA340F8
:10A3D000A140DB430C00122807D80849920052180C
:10A3E000116819402143116030BD054A11680B40C6
:10A3F00023431360F8E7C04687C0001108F000400F
:10A4000014F00040C21F70B5D4B20623092C0BD83B
:10A410000125084C9540002908D00021FFF7CAFF0C
:10A4200023682B4323600023180070BD2368AB43CF
:10A43000F8E7C04600380040214BF0B51B185B78A8
:10A44000022B21D1032444431E4A1F4EA35C121940
:10A450009478012215008540B76B013CE4B23D437E
:10A46000A240B563194C122815D89B0000290CD1C5
:10A4700017495B1899680A439A600123205C154AC2
:10A48000834011680B431360F0BD11495B18996854
:10A4900091439960F1E70E4B00290DD159690A43A8
:10A4A0005A61225C1328E8D00123203A93400A49DC
:10A4B000086803430B60E7E7596991435961F0E786
:10A4C0006466FF1F87C0001100800040CCC00011EF
:10A4D00000F00040A0F00040A4F00040F8B50024D7
:10A4E0001B4E1C4D1C4B1B5D012B1FD1194A926941
:10A4F000E2401A420BD00122B25693402200143A95
:10A50000D2B2022A09D815494A6913434B61013472
:10A5100002360C35172CE5D1F8BD0022B2560F4992
:10A520009200521891680B439360F0E7022BEED132
:10A53000E7B23800FFF71EFF01235840C1B23800D0
:10A54000FFF77AFF3800FFF715FF6877DFE7C046AF
:10A5500059C000116466FF1F6566FF1F00F00040D0
:10A56000012202388240054B002903D059690A4371
:10A570005A617047596991435961FAE700380040C0
:10A58000F8B50E0001210F008740114A0400D3687E
:10A59000FD43BB43D360831E8B4201D8FFF7E0FF2E
:10A5A00000212000FFF72EFF0A4A0B4B5168012EB5
:10A5B00005D139431B1951605E700020F8BD294058
:10A5C000516002221C1962709A6915409D61F4E77E
:10A5D00000380040008000406466FF1F012210B573
:10A5E0008240074B002906D019680A431A600121EE
:10A5F000FFF7C6FF10BD196891431960F7E7C04621
:10A60000008000400C2370B5002543430A4A29000E
:10A610009B181D70094B04001B185D70FFF7B0FFFD
:10A620000123A340064928000A681A430A60054925
:10A630000A689A430A6070BD8066FF1F6466FF1F48
:10A64000348000403080004070B504000E00FF28C8
:10A6500013D003250540FFF7D5FF084AA3089B0048
:10A660009B183F22ED00AA40AE401968200091439C
:10A67000314319600121FFF78DFE70BD183800408D
:10A68000F8B50C244443134B0500E4186368002B11
:10A6900003D1A3681220002B1AD0022201270E4BEF
:10A6A00000215B195A7028002770FFF769FF636863
:10A6B0001E1E08D0A3683E00002B04D02800FFF720
:10A6C00059FE4640F6B228003100FFF709FE00208F
:10A6D000F8BDC0468066FF1F6466FF1FF7B5C42043
:10A6E000FF222B4B80001958002491433F3A0A4324
:10A6F0001A508022274F5202274E1A60274B1D5DA9
:10A70000002D21D0A31E012B03D80121E0B2FFF7B9
:10A7100027FF012D18D11F4B9B69E3402B4213D01B
:10A72000E3B218000193FFF725FE01000198FFF73F
:10A7300055FFE3B2143B022B1DD801217156184A74
:10A740008D405369AB4353613B7F002B0DD0E5B285
:10A750002800FFF795FF2800FFF70CFE7B7F010024
:10A76000834202D02800FFF7A5FD01340C370236E2
:10A77000172CC3D1F7BD012100237156F3568D402C
:10A78000074A9B009B189A68AA439A60DCE7C04678
:10A7900000E100E06466FF1F59C000116566FF1FFD
:10A7A00000F0004010B501210400FFF7E9FE01238D
:10A7B000044A002011194B70A34091690B43936127
:10A7C00010BDC0466466FF1F70B50E001500040082
:10A7D000FFF718FF0C236343094A20009B189D6074
:10A7E0005E60FFF74DFFF021064B074A8900051E0A
:10A7F0005A5002D02000FFF705FF280070BDC04668
:10A800008066FF1F0000FF1F11A3001170B5134DDC
:10A8100007202C78002C1FD19822210052002800FC
:10A8200001F002FA0123C420FF222B700C4B8000A0
:10A830001C635C630B4B1C605C600B4B19589143B1
:10A840003F3A0A431A50802252021A600D20074AEA
:10A85000074901F059FA200070BDC0466466FF1F29
:10A8600000800040A0F0004000E100E0DDA6001103
:10A87000DDA40011030010B50620072B09D8054AF6
:10A88000137001F089F9D7210020034B034A890096
:10A890005A5010BDA443FF1F0000FF1FC91BFF1F1C
:10A8A00070B51D0002240C2910D8094ACA40D207ED
:10A8B0000CD5FBF72FFF041E08D1059A0499280038
:10A8C000FBF744FFFCF7B2FDFFF712FB200070BD61
:10A8D0001210000030B50D7802232C009C43184262
:10A8E00001D02B431C0008252300AB43284201D094
:10A8F0002B00234320241D00A543204201D01C43EC
:10A9000025002A230D70184204D011781E3B0B43FA
:10A91000137030BD0028FCD10C2113788B43F7E76E
:10A92000F8B51D0006AB1B88140007AA0E000B200B
:10A930001778002B27D10A78022A49D14A68507823
:10A9400011780002244A08438018042840D801F0F6
:10A950002BF803121D1B2300F06801F035F8021CD0
:10A96000C0B2B84200D93A1CD2B22000F1682A80A5
:10A9700000F06AFF06E00222F3681B882A80237039
:10A980001B0A63700020F8BD0622EEE701232B802E
:10A99000F3681B782370F5E7F368002B16D00822C4
:10A9A0002A801A8822701A88120A62705A88A27045
:10A9B0005A88120AE2709A8822719A88120A627181
:10A9C000DA88A271DB881B0AE371DBE72B80D9E709
:10A9D00001202B80D7E7C04600D6FFFFF7B5160051
:10A9E0000A781D0008AB1F880C000123022A18D129
:10A9F0004A685078117800022B4A084380180328CF
:10AA00000FD800F0D1FF02254439E06800F0DCFFE8
:10AA1000C0B20723B84204D37B190193152B02DD82
:10AA20000D231800FEBDE0682A003100C01900F0B7
:10AA30000BFF6B4600209B88E268D0541B4B1B68C1
:10AA4000834203D01B68834200D098470023E8E785
:10AA50000B23002FE5D1022DE2D1737832781B024F
:10AA60001343E2681380114B1B68002BEED01B6868
:10AA7000002BEBD00120E8E70B23002FD1D1062DCE
:10AA8000CED12A003100E06800F0DEFEDEE70B23C5
:10AA9000002FC6D1012DC3D132787533012AC0D819
:10AAA000E3681A70D2E7C04600D6FFFF7068FF1F48
:10AAB00070B50C001500072837D800F075FF041496
:10AAC00036361B36242E182015290BD8184E162280
:10AAD0000021300001F020F922002900300000F0B0
:10AAE000B3FE002070BD18200229FBD11288114B43
:10AAF0001A80F6E718200829F4D10A000E48290028
:10AB000000F0D2FFEDE718200129EBD10B4B1078B4
:10AB10000B49DA69FFF7DEFEE3E718200129E1D1EE
:10AB2000064B10780749DA6BF4E70220DAE7C046F3
:10AB30005868FF1F2244FF1F1844FF1FA843FF1F30
:10AB4000D043FF1FF043FF1F030010B50020DB07B9
:10AB500004D50721024A034800F08CF810BDC04616
:10AB6000E4C00011A843FF1F054A03001068002835
:10AB700003D082889A4201D1806870470068F6E766
:10AB8000686AFF1F0A88030008009A4204D08A8876
:10AB900004309A4200D0002070470000F8B5F2223D
:10ABA00000230D4F0D4E79680500424333709942E2
:10ABB00000D07B600A4C0021200001F0ADF800239A
:10ABC0001A007C60AB4202D100203370F8BD013323
:10ABD0002280DBB2F234F5E7606BFF1F5E6BFF1F74
:10ABE0006C6AFF1F73B56B4601900600684615003E
:10ABF0001980FCF74DFF041E11D1002D0FD076896E
:10AC0000002E11D00C2000F0BFFF00280ED0084A03
:10AC10000460136886808560002B02D110602000DC
:10AC200076BD1A001B68F7E70224F8E71324F6E75D
:10AC3000686AFF1F012100220A4B10B549420A4CE5
:10AC4000198099809A719A70084B207001201980A0
:10AC50005A60FFF7A3FF2078FCF778FF0448FDF760
:10AC600033FF10BD7868FF1F686BFF1F606BFF1F0D
:10AC700021AD0011022310B5002802D0FFF7B2FF6A
:10AC80000300180010BD0000030010B50020DB0712
:10AC900004D50421024A0348FFF7A4FF10BDC046B3
:10ACA000F8C000112844FF1FF0B50E2687B00393AB
:10ACB0000CAB1F8802ABF6180500080031000292A9
:10ACC000FDF768F804000120002C0FD03088FFF752
:10ACD0004BFF03000E20002B08D05E68002E05D02D
:10ACE00021002800039B029A0097B04707B0F0BDEF
:10ACF0000A4B10B5984207D10122002352420A8024
:10AD00008B708A808B7110BDFFF73CFF0028FAD052
:10AD100001235B42038000238370F4E7FFFF000000
:10AD2000F8B5050001290AD1134E00243388F22713
:10AD3000AB4219D028001149FFF7DAFF06E00229DB
:10AD400004D10139FDF73EFF0028EDD0F8BD3B00EE
:10AD500063437268D018D35A002B09D03A000021FF
:10AD600000F0DAFF0134E4B2054B1B78A342EED8C1
:10AD700001235B423380DDE7606BFF1F7868FF1FB4
:10AD80005E6BFF1F10B5FFF7FDFE0300002083423E
:10AD900000D0987810BD0000F0B589B01C000EAB53
:10ADA00080CB03901E8810AB1B78049202930B7A21
:10ADB0000D00DB0616D42B780593022B24D00498C3
:10ADC000FFF7D2FE002812D003689C46002B0ED05D
:10ADD000029B2200019329003B00644603980096E1
:10ADE000A04705E00498FFF7BFFE002802D10E201F
:10ADF00009B0F0BD8368002BF9D00A22290003981E
:10AE000098470028D7D0F3E76B6858781A786B4BCF
:10AE1000000210439842D2D8043B984210D2684BAB
:10AE2000984242D015D8674BC0180128C7D80B20CC
:10AE3000002EDDD1EB681A7859683A80200028E0AE
:10AE4000614BC018032800D979E000F0ADFD846A99
:10AE5000789E5E4B9842B2D10B20002EC8D10123C0
:10AE60003B80EB6831001B7823706889013080B229
:10AE7000FCF790FF3A88031E0ED0017802328A1840
:10AE80003A80428962704289120AA2705968027837
:10AE9000E01C00F0D9FC06E004323A8031000422C4
:10AEA000601C00F039FF0020A2E70B20002E9FD18C
:10AEB000EB6807A91E8804233B80330A3000267004
:10AEC0006370FCF767FF051E28D004AB9A890E2338
:10AED00004A95B183E49C668FCF7D0FF00280BD1D7
:10AEE0002B783C486A680599FBF786FB002803D15C
:10AEF000012304AA5B42D3813278022A06D1716809
:10AF0000201D00F0A1FC3B8802333B800E2304AAE5
:10AF10009B181B88A3701B0AE370C4E704ABDE8197
:10AF2000F4E70B20002E00D062E7E9680398FFF7F2
:10AF300029FF02233B802070000A6070B3E70B20DA
:10AF4000002E00D054E70222EB681B883A80237061
:10AF50001B0A6370A7E7E86800F036FDC2B2030081
:10AF60000720B24200D243E70DD00299DBB271183C
:10AF7000994202DB921BD3B20293029BE9681A004A
:10AF80003B8089195AE70023F6E70B20002E00D0FA
:10AF90002EE70722EB683A801A7822705A7862709E
:10AFA0005A88A2705A88120AE2701A792271DA88D5
:10AFB0006271DB881B0AA37175E7C0460429000093
:10AFC0000228000000D8FFFFFFD6FFFF0328000083
:10AFD000FFFF000028C00011F0B58DB06B460020C7
:10AFE000089120229B5E83423DDAA64B187800F040
:10AFF0000BFE071E32D00378B02B2CD1007902381B
:10B0000016281FD800F0B8FB17001E001E001E00F7
:10B0100031001E0096001E001D011E0052011E0080
:10B0200073011E00CD011E0050021E001E001E00F6
:10B030008E021E00E302944B94491B8878880B8093
:10B04000FBF71AF83800FCF79BFF914B1B68002BAD
:10B0500001D038009847380000F08EFD8020089B12
:10B060000002434018000DB0F0BDEE2200218748D9
:10B0700000F052FE0BAA3B7B7989388900923A0096
:10B080000D32FCF79FFD0400804B1B78002C3FD154
:10B0900046E0804B788805937F4B4100CB5A0BAE3E
:10B0A000073BDBB232880293002301937B4B2100E4
:10B0B00006930093059BFFF76FFE744D002810D197
:10B0C000069B3A8A1B889A420BD1380005991230A8
:10B0D00000F0E2FB002804D02B7862899B00EB187B
:10B0E0005A80162306A81B18328820007989FCF79D
:10B0F000C5FE2B7804009A00AA1851880029C3D0F5
:10B100000133DBB22B70002807D006A9C98A9180D1
:10B11000634A12889A42BCD802E0012149429180D8
:10B12000002B04D059497888FAF7DAFF8AE73E897C
:10B130000A2479E000253E89574B06937B88069ABE
:10B140005B009B5A033B9D4202DB002DF0D05BE08D
:10B15000162206A812183B7B798900923A0030002B
:10B160000D32FCF72FFD0590002858D04689017A52
:10B170007888FCF7F1FC041E44D1464B788807938D
:10B18000069B4100C95A454B0439C9B206AAD28A66
:10B1900006930291019400930599079BFFF7FCFD2C
:10B1A000041E2FD1069B39491A88931C002D26D1E5
:10B1B0004B807988384B4900CB5A5119033B8B425D
:10B1C00020DD059B31485B8941190B71A91C0135B4
:10B1D000C9B2EDB2059145191B0A2B71059B2D498A
:10B1E0000433181800F030FB2C4B059A1B88D31839
:10B1F000DDB22C4B9E4205D00136B6B29CE74988A1
:10B200009942D6D0002D0CD0204C2800618800F047
:10B210006BFC207021007888FAF772FF12E7059C1A
:10B22000F0E7002C00D183E77B78142B00D109E7ED
:10B2300016493B794E800B700C717888FAF712FF33
:10B2400000E7162406ABE41821003889FCF7A2FDBC
:10B25000011E00D1B7E1788822880F4C45002C5B95
:10B260000A4D013CE4B2029400240F4B0194009576
:10B27000FFF792FD041E00D014E129007888FAF748
:10B280004FFFDFE6686BFF1F1443FF1F8068FF1F3F
:10B290007468FF1F7469FF1FB064FF1F646AFF1F9B
:10B2A0001243FF1FFFFF00008268FF1F162406AB3A
:10B2B000E41821003889FCF76DFD011E00D182E100
:10B2C00078882288AE4C45002C5BAE4D013CE4B240
:10B2D00002947C89AC4B01940095FFF75DFD041E40
:10B2E00000D0DFE029007888FAF724FFAAE60025DD
:10B2F000A44B1D803B00F6331B78A24A7888079246
:10B30000AB4208D99E4B12880693069943005B5ABC
:10B31000013B9A4203DB0799FAF716FF92E61624DF
:10B320006B00FB18059306ABE418059B21001889F8
:10B33000FCF730FD011E03D1059B01241E8973E734
:10B340007888924B2288069C099343001B5B904EA1
:10B35000013BDBB20293002300960193099BFFF7A8
:10B360001BFD041E02D0059B1E895DE77B88069AA3
:10B370005B009B5A079A108832881218934202DCAD
:10B380001B1A013B33807F4C023032880999001927
:10B3900000F05AFA2388328801359B182380EDB2D9
:10B3A000A8E70BAA3B7B7989388900923A000D32D5
:10B3B000FCF708FC00250590059B002B04D10A240E
:10B3C000002D00D16EE060E0059B7888197AFCF7CB
:10B3D000C3FB0100041E63D1694C6C4B7888069452
:10B3E0000993069B4400E45A694B063CE4B20BAE59
:10B3F000328807930294019100930599099BFFF706
:10B40000CBFC041E4CD1079B5E491B881A1D002DE6
:10B4100030D14A80059B5B4C5A8963191A716B1CA9
:10B420009BB2E318120A1A71162306A832881B1859
:10B4300079890598FCF722FDFF21AA1C2E1D0335F2
:10B440000B00059092B2B6B2ADB2002803D006ABA5
:10B45000DB8AD9B21B0AA218651911712B714C4DE8
:10B46000301D2A884949201800F0EEF92B88F6187B
:10B47000B5B2A1E74988914207D17A88069952006E
:10B48000525AEB18053A9A42C4DC3E4C28006188B7
:10B4900000F07AFC207021007888FAF75FFED1E591
:10B4A000002DF2D13E89BFE6162606ABF618310014
:10B4B0003889FCF76FFC3D000400FA3500282DD0D8
:10B4C000037A9B060CD400227B8939897888009204
:10B4D0003A000C32FFF7E8FB041E10D03E8915E05D
:10B4E0003088FFF741FB00281AD08368002B17D063
:10B4F0002100122278889847041EE4D0EEE72B78CA
:10B50000002B02D17888FAF739FE00262B78002B21
:10B5100000D097E5002C00D194E585E60124DDE715
:10B520000E24DBE7162506ABED1829003889FCF759
:10B5300031FC041E47D0037A9B0611D4154A7B8840
:10B540001188994203D01448814207D11380134BCC
:10B55000F2261D780023D9B2A94221D30924A1E7FC
:10B560002888FFF701FB00282FD08368002B2CD000
:10B570002100122278889847041EDFD092E7C04647
:10B58000B064FF1F8068FF1F8268FF1F7469FF1F80
:10B59000646AFF1F606BFF1FFFFF00005E6BFF1FF1
:10B5A00031005943546801336018615A0029D2D1DF
:10B5B0003C0008342100F22200F046F9210078888E
:10B5C000FAF7E4FD3EE501246CE70E246AE71D4B23
:10B5D0001A887B889A4231D07888FAF7E1FD31E504
:10B5E000F223059851684343CD18C95A00291FD04A
:10B5F0003B7A012B0BD16C88AB887888AA1D00940C
:10B60000FFF752FB041E02D000233B722E88F22269
:10B610000021280000F080FB00232B80059B0133D4
:10B62000DBB20593084B05991B78064A8B42D7D8A5
:10B6300001235B421380002CCED0F5E500263400B8
:10B640000596EFE7606BFF1F5E6BFF1F70B5040090
:10B650000E001500FFF796FA031E08D131000548C9
:10B66000FFF790FA03001120002B02D01C8000206D
:10B670009D7070BDFFFF0000F8B50B4F06003B78D2
:10B680000D001400FF2B0ED00A2000F0FDF9011E62
:10B6900009D0B1230380002346800371C580048153
:10B6A000387800F0A9F8F8BD6944FF1FF7B50F001E
:10B6B00008A90600088809A90B240988002821D1B7
:10B6C0000234022B1ED1557813782D021D432B0016
:10B6D0008B4301937334002B14D1FB6830001900A5
:10B6E0000093FFF74FFB019C85420BD02A003000EE
:10B6F0000099FFF7ABFF041E04D12A0030007989BE
:10B70000FFF7BAFF2000FEBDF0B50E7885B00390BC
:10B710000AA805880120022E0DD14C68277864788C
:10B7200024023C43054FBC4205D10398DBB201968D
:10B730000095FFF7BBFF05B0F0BDC0460229000031
:10B74000034B10B51B68002B00D09847FEE7C0469E
:10B750006C6BFF1F07B501A8FFF7F2FF044A05480D
:10B760000021121A00F060FAF8F786F8FEE7C046EA
:10B77000706BFF1F6C44FF1F01B40248844601BC7C
:10B78000604700BF853BFF1F01B40248844601BCEF
:10B79000604700BF3555000001B40248844601BC33
:10B7A000604700BF2951010001B40248844601BC32
:10B7B000604700BFF30E000001B40248844601BC9C
:10B7C000604700BF413BFF1F01B40248844601BCF3
:10B7D000604700BFE117000001B40248844601BC85
:10B7E000604700BF3119FF1F01B40248844601BC05
:10B7F000604700BF8D12000001B40248844601BCBE
:10B80000604700BF594F010001B40248844601BCA3
:10B81000604700BF691F000001B40248844601BCB4
:10B82000604700BFED3AFF1F01B40248844601BCE7
:10B83000604700BFD91B000001B40248844601BC28
:10B84000604700BFC130FF1F01B40248844601BCFD
:10B85000604700BFE94C010001B40248844601BCC6
:10B86000604700BF7918000001B40248844601BC5B
:10B87000604700BFB54C010001B40248844601BCDA
:10B88000604700BF055E000001B40248844601BC69
:10B89000604700BF9D36FF1F01B40248844601BCCB
:10B8A000604700BFCD4C010001B40248844601BC92
:10B8B000604700BF5147010001B40248844601BC03
:10B8C000604700BF2146010001B40248844601BC24
:10B8D000604700BFC521000001B40248844601BC96
:10B8E000604700BF2526000001B40248844601BC21
:10B8F000604700BF1D4B010001B40248844601BCF3
:10B90000604700BF056A000001B40248844601BCDC
:10B91000604700BF9137FF1F01B40248844601BC55
:10B92000604700BFF919FF1F01B40248844601BCFB
:10B93000604700BFEDA5000001B40248844601BC89
:10B94000604700BFC56D010001B40248844601BCD8
:10B95000604700BF8B52010001B40248844601BC1D
:10B96000604700BF5522000001B40248844601BC74
:10B97000604700BFC51D000001B40248844601BCF9
:10B98000604700BF0519FF1F01B40248844601BC8F
:10B99000604700BFADAE000001B40248844601BC60
:10B9A000604700BF5934FF1F01B40248844601BC00
:10B9B000604700BF713BFF1F01B40248844601BCD1
:10B9C000604700BFA930FF1F01B40248844601BC94
:10B9D000604700BFDD52010001B40248844601BC4B
:10B9E000604700BFC926000001B40248844601BC7C
:10B9F000604700BFE932FF1F01B40248844601BC22
:10BA0000604700BF4550000001B40248844601BCB5
:10BA1000604700BFD949010001B40248844601BC17
:10BA2000604700BF9136FF1F01B40248844601BC45
:10BA3000604700BFC539FF1F01B40248844601BCFE
:10BA4000604700BF1147010001B40248844601BCB1
:10BA5000604700BF713AFF1F01B40248844601BC31
:10BA6000604700BF350E000001B40248844601BCA7
:10BA7000604700BF4D39FF1F01B40248844601BC36
:10BA8000604700BFC94A010001B40248844601BCB6
:10BA9000604700BF1D4D010001B40248844601BC4F
:10BAA000604700BFED4A010001B40248844601BC72
:10BAB000604700BF810E000001B40248844601BC0B
:10BAC000604700BF8539FF1F01B40248844601BCAE
:10BAD000604700BF5549010001B40248844601BCDB
:10BAE000604700BF193BFF1F01B40248844601BCF8
:10BAF000604700BF350E000001B40248844601BC17
:10BB0000604700BFB352010001B40248844601BC43
:10BB1000604700BFE548000001B40248844601BC0C
:10BB2000604700BF3D18000001B40248844601BCD4
:10BB3000604700BFB14E000001B40248844601BC1A
:10BB4000604700BF090E000001B40248844601BCF2
:10BB5000604700BF456B010001B40248844601BC48
:10BB6000604700BF2124000001B40248844601BCA4
:10BB7000604700BF3939FF1F01B40248844601BC49
:10BB8000604700BF434D010001B40248844601BC38
:10BB9000604700BF3D4B010001B40248844601BC30
:10BBA000604700BFC91BFF1F01B40248844601BCA7
:10BBB000604700BF5952010001B40248844601BCED
:10BBC000604700BFDD66010001B40248844601BC45
:10BBD000604700BF4551010001B40248844601BCE2
:10BBE000604700BF4538FF1F01B40248844601BCCE
:10BBF000604700BFC9A9000001B40248844601BCE7
:10BC0000604700BFC136FF1F01B40248844601BC33
:10BC1000604700BFF54E010001B40248844601BCF4
:10BC2000604700BF053AFF1F01B40248844601BCCB
:10BC3000604700BFB70E000001B40248844601BC53
:10BC4000604700BFF94C010001B40248844601BCC2
:10BC5000604700BF2933FF1F01B40248844601BC7E
:10BC6000604700BFE928000001B40248844601BCD7
:10BC7000604700BF6DBC000001B40248844601BCAF
:10BC8000604700BF091B000001B40248844601BCA4
:10BC9000604700BF311B000001B40248844601BC6C
:10BCA000604700BF5D17000001B40248844601BC34
:10BCB000604700BF014C010001B40248844601BC4A
:10BCC000604700BF5125000001B40248844601BC12
:10BCD000604700BF75A9000001B40248844601BC5A
:10BCE000604700BF0124000001B40248844601BC43
:10BCF000604700BF291C000001B40248844601BC13
:10BD0000604700BF017F000001B40248844601BCC7
:10BD1000604700BF4931FF1F01B40248844601BC9F
:10BD2000604700BF154D010001B40248844601BCC4
:10BD3000604700BF6571010001B40248844601BC40
:10BD4000604700BF9DA9000001B40248844601BCC1
:10BD5000604700BFA54F010001B40248844601BC02
:10BD6000604700BF4D1F000001B40248844601BC7B
:10BD7000604700BF0D52010001B40248844601BC77
:10BD8000604700BF851F000001B40248844601BC23
:10BD9000604700BF090E000001B40248844601BCA0
:10BDA000604700BF156B010001B40248844601BC26
:10BDB000604700BF5D3BFF1F01B40248844601BCE1
:10BDC000604700BFA946010001B40248844601BC97
:10BDD000604700BF692EFF1F01B40248844601BCC2
:08BDE000604700BF855201001D
:10BDE800000101030202030304030502060207021D
:10BDF800080209030A030B030C020D000E030F03CC
:10BE0800100311031303140315001600493C001115
:10BE18007D3C001100000000020000002ABE001155
:10BE2800192A0F180A000000F1590000FD2400002B
:10BE380041460100D1810011E5A1001139760011B8
:10BE4800D57F001179540011D9AF0011C5500011E8
:10BE5800593E0011893F001100000000161600002D
:10BE68000200000074BE0011F4FFF3FFD2FC0000D2
:10BE7800C9400011000000000000000054757961FD
:10BE88000042322E300030303135006769746875F1
:10BE9800622E636F6D2F70767678005448303500C7
:10BEA80002000000BCBE0011292A282A272A262AB7
:10BEB800252A242A0A180000E20400007102000062
:10BEC80078EC000005000000744000001027000016
:10BED80060F000000400000006640000204E00002E
:10BEE80000000000060000005C440000102700006D
:10BEF8006CEE000007000000050000001F501D1038
:10BF0800023CB4000001150020000000A10200005E
:10BF18003031323334353637383941424344454677
:10BF2800000000007D580011D158001100000000E9
:10BF38000200000044BF00116F2A6E2A1A18EAD8BE
:10BF4800BC80F0FC60000000000000000000F3036B
:10BF5800B59747D6F613F7D777E6F0A7F47400003D
:10BF680001A00000000000006410B71DC8206E3B4F
:10BF7800AC30D9269041DC76F4516B6B5861B24DE8
:10BF88003C7105502083B8ED44930FF0E8A3D6D652
:10BF98008CB361CBB0C2649BD4D2D38678E20AA0BA
:10BFA8001CF2BDBDFB349B5F8000008000100000C8
:10BFB800000000003B620011C57800115F620011AB
:10BFC800CD7C0011E3620011A37C001159630011BC
:10BFD800797C0011AB630011417E001113640011DC
:10BFE800417E001145640011FB7D00115963001169
:10BFF800317C0011D1630011D97D001100000000CF
:10C0080000000000B7640011D97D00111965001106
:10C01800DD780011052A042A012A002A02290328AA
:10C028000128002801180018000000000000000086
:10C038000000000000000087010102010201010266
:10C0480001020303040103010101010103030201C9
:10C0580003000D000E001000110013001401070169
:10C0680008010A010B011C011D0204020502070256
:10C07800080219021A021C021D0301030203170019
:10C088000201000504000807000B0A001716001D2E
:10C098001C010201010504010E0D01111001141308
:10C0A800011716011A19020201020B0A020E0D02EB
:10C0B8001110021413021716030504030807030BD3
:10C0C8000A030E0D0001020307090A0B0E0F1011D7
:10C0D80012141718191A1B1F2021220021A9001158
:10C0E800DDA9001100000000020000002EC00011B0
:10C0F8000000000009B70011000000000200000065
:04C108002CC0001136
:020000041FFFDC
:1000000000000000C13D001130BE00112CBE0011E7
:100010009C61FF1F000000000000000000000000C5
:1000200000000000000000000000000000000000D0
:1000300000000000000000000000000000000000C0
:1000400000000000000000000000000000000000B0
:1000500000000000000000000000000000000000A0
:100060000000000000000000000000000000000090
:100070000000000000000000000000000000000080
:100080000000000000000000000000000000000070
:100090000000000000000000000000000000000060
:1000A0000000000000000000000000000000000050
:1000B0000000000000000000000000000000000040
:1000C0000000000000000000000000000000000030
:1000D0000000000000000000000000000000000020
:1000E0000000000000000000000000000000000010
:1000F0000000000000000000000000000000000000
:1001000000000000000000000000000000000000EF
:1001100000000000000000000000000000000000DF
:1001200000000000000000000000000000000000CF
:1001300000000000000000000000000000000000BF
:1001400000000000000000000000000000000000AF
:10015000000000000000000000000000000000009F
:10016000000000000000000000000000000000008F
:10017000000000000000000000000000000000007F
:10018000000000000000000000000000000000006F
:100190004D33FF1F9531FF1FC166010000000000B5
:1001A000000000000000000000000000000000004F
:1001B000000000000000000000000000000000003F
:1001C000000000000000000000000000000000002F
:1001D000000000000000000000000000000000001F
:1001E000000000000000000000000000000000000F
:1001F00000000000000000000000000000000000FF
:1002000000000000000000000000000000000000EE
:1002100000000000000000000000000000000000DE
:1002200000000000000000000000000000000000CE
:1002300000000000000000000000000000000000BE
:1002400000000000000000000000000000000000AE
:10025000000000000000000000000000000000009E
:10026000000000000000000000000000000000008E
:10027000000000000000000000000000000000007E
:10028000000000000000000000000000000000006E
:10029000000000000000000000000000000000005E
:1002A000000000000000000000000000000000004E
:1002B000000000000000000000000000000000003E
:1002C000000000000000000000000000000000002E
:1002D000000000000000000000000000000000001E
:1002E000000000000000000000000000000000000E
:1002F00000000000000000000000000000000000FE
:1003000000000000000000000000000000000000ED
:1003100000000000000000000000000000000000DD
:1003200000000000000000000000000000000000CD
:1003300000000000000000000000000000000000BD
:1003400000000000000000000000000000000000AD
:10035000000000000000000000000000000000009D
:10036000000000000000000000000000000000008D
:1003700055B7001100000000000000000000000060
:10038000000000000000000000000000000000006D
:10039000000000000000000000000000000000005D
:1003A000000000000000000000000000491BFF1FCB
:1003B000000000000000000000000000000000003D
:1003C000000000000000000000000000000000002D
:1003D000000000000000000000000000000000001D
:1003E000000000000000000000000000000000000D
:1003F00000000000000000000000000000000000FD
:08183800706FFF1F4118FF1F34
:10184000024981F3088802F0EFFB0000706FFF1F70
:1018500070B500241E491F4A1F484C6308CA1B0567
:101860001B0DE4188242F9D11C4B80228B630021AE
:1018700009201B4B920519621A4B1B4DDA671B4B53
:10188000DA688243DA609A68194802409A60112047
:10189000296002F0B7F8112002F094F880226B6CF6
:1018A000112093436B64EE23DB006343114A1B0C4E
:1018B00013840122104B9A7201F022FC0F4B1B780B
:1018C000002B04D10E4B1021187802F0C5F970BD21
:1018D000000005408805054000060540FF010000A6
:1018E00000F0004004E100E0003800403CF000401F
:1018F000FFDFFFFF6C61FF1F2062FF1F4E64FF1FB1
:101900004C62FF1F10B502F067F9072804D01228B7
:1019100008D0022808D010BD044A0420136B0133FC
:101920001363F8E70220F6E71420F4E75865FF1F79
:10193000F8B507000C0026002500503630785135E8
:10194000002804D10300287058342370F8BD29788A
:10195000CA00481E8141A3183800A25C5B68C9B266
:10196000FFF7D0FF00280DD12B78DA00A218013341
:1019700050602B703378044A013B3370136A013393
:101980001362D8E70123DFE75865FF1F5C23434359
:10199000074910B5C9180B0058331B78012B05D126
:1019A000FFF7C6FF034A936A0133936210BDC04636
:1019B0008C65FF1F5865FF1F10B502F08DF9064AB0
:1019C0000121130010CB4942D967044B136002F088
:1019D000FBFA200010BDC04600E100E0100010003E
:1019E00010B5040002F078F9024B1C6002F0ECFA2A
:1019F00010BDC04600E100E010B5040002F06CF933
:101A00004021094A200013688B43136000F0F6FA66
:101A100001F07EFC0022054B01201A60044B0432C9
:101A20001A6002F0F1F8FEE71CF00040C4F000403C
:101A3000C0F00040431E5A425341A022F0B5D201EB
:101A40005B421340154D164A40019B182A18127E1E
:101A50008BB00191002A1BD01A000832D46F0022EB
:101A6000E6B206AFE4B294420EDC2818C369002B3C
:101A700008D0019902AA117106AA049202AA16734B
:101A800003A898470BB0F0BD1978B9540132EAE7C2
:101A90001A7D1A7806AB01261A70E6E71868FF1F50
:101AA00000400040F0B5254B04004001C25C85B009
:101AB000002A2BD01A18117E002927D0917E0029E8
:101AC00024D01179022921D11689D788D168F51B34
:101AD000ADB22A1C102D00D9102292B2BE4217D1ED
:101AE0001818012303710023C269C38003819A423D
:101AF00006D06846032103730171029301A8904741
:101B00000820002C00D0192001F0FAFA05B0F0BD31
:101B1000013C65426C41A0256442ED012C40084D1A
:101B20001B186419074D0633013A92B2AA42EDD050
:101B30001888461C1E80085C2070F5E71868FF1F97
:101B400000400040FFFF00000F220E4B10B59868C8
:101B5000104002380A280BD802F00AF80D0A0B0AC6
:101B60000A110A0A0A0A060002210020FFF762FF92
:101B700010BD0121F9E70020FFF794FFF8E7DB6FC4
:101B8000F6E7C046004000400F220E4B10B59868A3
:101B9000104002380A280BD801F0EAFF0E0A0B0A9F
:101BA0000A120A0A0A0A060002210120FFF742FF70
:101BB00010BD01210800F9E70120FFF773FFF7E7E7
:101BC000DB6FF5E70090004013B5334C2378072B0B
:101BD0003DD8324B1A78324B002A39D1802219680D
:101BE00052020A431A60252001F0CCFE20232D4A20
:101BF00011680B43802113606B460422C9050868F5
:101C00000733104228D080210422C905C868104239
:101C10002ED080212020C905CA688243CA601422C0
:101C20001A701A78002A2FD18021C905C86820327D
:101C30000243CA6014221A701A78002A28D11A4B5B
:101C40001A7D22785A601D221A705932DA6013BD4B
:101C50001A6816490A40C5E7086802430A60142258
:101C60001A701A78002ACED01A78013AD2B2F7E761
:101C7000C8680243CA6014221A7019784A1ED2B288
:101C80001A700029F9D1C4E71A78013AD2B2C7E72D
:101C90001A78013AD2B2CEE7A443FF1F6C44FF1F6B
:101CA0003CF000409C43FF1F00200040FFFFFEFF70
:101CB000564B70B51B68012B03D1554A936D013308
:101CC000936502F099F8534B534A1860534B544CA8
:101CD0001A600123534A1360534A13602378002B80
:101CE00006D006225149524802F026F900232370FB
:101CF000504A514B10681B78C1B2002B0ED14F4C8B
:101D0000C0B223785BB2002B4FDB237824785BB220
:101D100064B21B0424021B191B1813600B1C5029EE
:101D20004ED95023464A47491078DBB2FF22022899
:101D30004BD10868444C454D267890432A7896420A
:101D400054D9227824782E78023B5D10A31B6B4374
:101D50005201D31A10335B111843086002F024F9C2
:101D6000031F012B45D83A4B1B78002B06D0394B6B
:101D70001B78002B02D0002002F0A6F8A122364BDF
:101D800092009978354B4A431B689B188322920036
:101D90009B181B78033B012B03D8AF20400002F0B7
:101DA00063F901222E4BDA8270BD237824785BB26E
:101DB00064B2FF33FF341B0424021B190138ABE764
:101DC000CAB2022AAED20223ACE70868254C264DDF
:101DD000267890432A78964208D9227824782D785C
:101DE000023B5B10641B63435201B2E72378DBB212
:101DF000B2E70228D5D11D4B1B78013B022B03D93A
:101E00001B4B1B78022BCCD16C20C8E79809FF1F15
:101E1000FC0FFF1FA464FF1FFF3F000014100340CE
:101E2000A864FF1F0C10034000100340D50BFF1FD8
:101E30007211FF1FB40003408C09FF1F680AFF1FC7
:101E4000490AFF1F94000340460AFF1F470AFF1F6D
:101E5000F908FF1F2209FF1F300DFF1F3409FF1F64
:101E6000BC0BFF1F440AFF1F450AFF1F1C09FF1F71
:101E70002309FF1F10B502F067F80022014B1A80FA
:101E800010BDC046A064FF1F10B501F0C5FEA12122
:101E9000054A89009478054A61431268044B521838
:101EA000528C1A8010BDC046300DFF1F3409FF1F31
:101EB000A064FF1F10B50D4B0D4A9978A1239B001C
:101EC0004B431268D218531DD97F0A4B1B88994285
:101ED00009D2441C07D0C82805D0D2695B1A5A43DE
:101EE000054B5343C01801F0A7FF10BD300DFF1F75
:101EF0003409FF1FA064FF1F7102000070B5244D5C
:101F00002B68002B28D001F0B7FF2B68D8402B6836
:101F10000400002B27D001F0F7FE2B68D8401D4BA2
:101F20001D4A9978A1239B004B431268D118D25CBB
:101F300091239B00002A20D0CA580132CA50174B67
:101F400017491B680868834214D3D23B181A012A28
:101F50001AD0144B186070BD01F08EFF124B196837
:101F600001F02AFFD3E701F0CFFE0F4B196801F013
:101F700023FFD4E70D495B18E8E7CA500C4B1B68F8
:101F8000DB68E418201AE4E7F530FF30E1E7C046EB
:101F90001C08FF1F300DFF1F3409FF1F9C09FF1F86
:101FA000A464FF1FA009FF1F1808FF1F2DFF3F009B
:101FB000AC64FF1F70B504000D00282916D1030082
:101FC000A433C2881B889B1A0B4A9BB293420DD93B
:101FD00006006A3605223100653001F08DFF0028C9
:101FE00004D13100200001F0C7FE70BD290020009F
:101FF00001F04AFEF9E7C046FE7F0000F8B5050093
:10200000012001F039FE134CA36AA26A9342FBD16E
:10201000114E336001F0A8FE10490300086010481B
:10202000426894460F4A17680022BC4501D24268B4
:10203000BA1A0D4802603268AD18A422E562606ADF
:10204000520302436262094A1278002A01D00F3B10
:102050000B60F8BD00F00040340AFF1FE408FF1FCA
:1020600028100040180AFF1F1C0AFF1F1C09FF1F31
:1020700070B580241025E405A3682B43A36001F00C
:1020800003FFA368AB43A36070BD0000F7B5160063
:1020900080221C001023D2050191916805000B439A
:1020A000936000225A4BD7301A6001F08DFD9D23BA
:1020B0002A002F009B00EB58CA3201210092FC3706
:1020C000002B01D00021009A386801F0D5FF2900CB
:1020D000009BCB311A784F4BD3351A604B780A7876
:1020E0001B0213438A7812041A43CB781B0613434E
:1020F000494A1BBA13604B790A791B0213438A7948
:1021000012041A43CB7931001B061343434A1BBA0E
:1021100013606B782A781B021343AA7812041A43BF
:10212000EB781B0613433E4A1BBA1360019A330235
:1021300013433C4A13603C4B22001B1B9C46032963
:102140003DDCB3089A0013005142B21A032A46D16B
:10215000354AE018511A827840781204000202438E
:10216000E05C043302430A600022FF2B4BDDF022C7
:102170002E4B12011A600F222D4B1A602D4A136844
:10218000002BFCD00023224A27491360091B321D73
:102190000B191B68043A180A23706070180C1B0E88
:1021A000A070E3700434002AF2DC802210213B6826
:1021B000D20501333B6093688B439360F7BD634660
:1021C000D578981893782D061B042B43157804397D
:1021D0002B43557804322D022B430360AFE7022ACC
:1021E0000AD1114AE05C511AE218527812020243F5
:1021F0000A6004339BB2B7E7012AB5D10A4A521AE2
:10220000E15C1160F5E7084959180A600433ACE74E
:10221000000004403C000440380004403400044006
:10222000300004400C00044000010440040004405D
:102230001000044014000440F7B5150080221C0073
:102240001023D2050091916807000B43936000238F
:10225000654AD730136001F0B7FC9D233E009B0018
:10226000F9583B00CA363200FC33002900D07FE029
:10227000586801F001FF390032785C4BCB311A60AD
:102280004B780A781B0213438A78AC4612041A432F
:10229000CB78281D1B061343554A1BBA13604B7994
:1022A0000A791B0213438A7912041A43CB791B065D
:1022B0001343504A1BBA13604B7A0A7A1B0213432A
:1022C0008A7A12041A43CB7A21001B0613434A4A26
:1022D0001BBA1360009A2B021343484A1360220072
:1022E000474B1B1B0093009BCE785B1801938B78A8
:1022F00036061B0433430E78043833434E780431DA
:1023000036023343019E33600328ECDC0321A80826
:10231000431C9B002940800003292BD13849E51834
:102320005E18A9786D78E35C09042D0229431943EE
:102330003160030008330021FF2B2DDD314B324982
:1023400019600F21314B1960012327490B60304B75
:1023500019680029FCD006211B680B40042B20D0F3
:1023600080220020D20593680A318B439360FEBD22
:1023700001217DE7022908D121495D18E11849783A
:10238000E35C090219432960D3E70129D3D11C4931
:102390005918E35C0B60CCE7194818180160043346
:1023A000CAE7002310490B606346002B0CDC3B009E
:1023B000FC335A68102101325A608022D20593689A
:1023C00001208B439360D2E7009B9B181B68190A7E
:1023D00013705170190C1B0ED37004235B42917063
:1023E0009C440432E0E7C046000004403C00044046
:1023F0003800044034000440300004400C00044025
:102400000001044004000440080F000010000440D4
:102410001400044070B5061E19D002225A4B9B7955
:102420009343012B13D1594B1A78FF2A0FD15A78B5
:10243000FF2A0CD19A78FF2A09D1DA78FF2A06D12F
:102440001A79FF2A03D15B79FF2B00D199E0504B19
:102450000C201A78012A08D000224E4D1A702978D3
:102460000B00093B042B01D8212070BD4B1F012B11
:10247000FAD9454CA37B042B00D982E0A279032A28
:1024800000D97EE09A1ED2B2012A02D860881F28A5
:1024900077D9002E56D0012E73D1A0880128E3D021
:1024A000002907D1581E032803D801F061FB121739
:1024B00015122E702978481E032811D80025364B96
:1024C0001D602823237501F0B7FDA84227D0A58001
:1024D000CAE702212970EDE70421FBE70321F9E7B0
:1024E00007390129C0D82D490968C96A8906BBD5B1
:1024F0002B4908780028B7D1012A01D9002BB3D184
:1025000002230B708021274D2633890128782375FB
:1025100001F062FD80212878890101F09DFB0123F3
:10252000A380214B1B78002B0AD0FA2280211F4B5D
:1025300092001B8809025A431A4B187801F074FC68
:10254000002092E701F0C8FB2B78A680073B012B07
:1025500003D917482E7001F077FB114B114C1A78F4
:10256000002A06D080210022207889011A7001F00B
:1025700033FD01F029FD80212078090201F02CFDB6
:10258000DEE7122071E7C046A60BFF1F6B09FF1F95
:102590001A09FF1F1C09FF1F4809FF1FAC64FF1F1A
:1025A0002309FF1F1B09FF1F2109FF1F2C09FF1F04
:1025B0000010004010B5002901D001F0B5FB10BD9E
:1025C000F7B5604B01919978A1239B004B435E4A7C
:1025D000060014681022E418D6235B00E058362366
:1025E000FF33E35C00279343222B41D1574B0F3A33
:1025F0001A600760012501F00FFC019B1880E82399
:102600005B00E35C002B01D0B34258DD0023504F48
:10261000FB70AD33FF33E3581A68002A03D09B8860
:10262000DB439B071DD03823FF33E35C002B18D01E
:102630009B235B00E35C002B13D1D133FF33E35CBE
:10264000B3420EDAA4235B00E15AE018090A023112
:1026500001F0DAFC23000122FE33013E01351A8726
:10266000FA70E8235B00E35C002B2AD0A8B2FEBD21
:1026700003683D00002BBED081880430090A023176
:1026800001F0C2FCD6235B00E3581F60B2E72300D1
:10269000B133BA00FF339858013781880430090AF2
:1026A000023101F0B1FCE8235B00E35CBB42EEDCED
:1026B000E822F61AED1800235200A354A6E70027DB
:1026C000F1E7200001F030FC00281FD0002E1DDDB6
:1026D0007319882647190193B600200001F09CFC6D
:1026E0005A30800020184068013581880430090A7A
:1026F000023101F089FC200001F04EFAA3590133A8
:10270000A351BD4202D0019B9D42E6D1114BE35C37
:10271000002BABD095239B00E35C002BA6D00E4B87
:10272000E15A0029A2D00D4AA35C994202D9013393
:10273000A3549BE700231A212000A35401F054FC6A
:1027400094E7C046300DFF1F3409FF1F00140340FB
:10275000E010FF1F5A020000720200005E0200003B
:102760000D4970B54A6E0D4CD2038B69D20BA24253
:1027700006D80B4D0224AA4204D901F08DFB70BD8E
:1027800002246442E21815007E2425402242F4D03F
:10279000A3432B438B61F0E700F000400A200000C8
:1027A000FC1C0000F8B51D4B1D4F1A78002A10D1F3
:1027B000BA7B002A02D101321A7003E0032AFAD050
:1027C000022AF8D001F038FC00220120154B1A70C3
:1027D000F8BD154B154D1C68154B9E7801232B70C9
:1027E0002878C0B200F09EFBBB7B002B0BD101F020
:1027F0000BFBA1239B007343E41883239B00E41885
:1028000023782B70E4E7032B02D101F0CDF9F0E738
:102810000020022BDCD101F017FCEAE71C09FF1FA6
:10282000A60BFF1F2309FF1F3409FF1F490AFF1FC3
:10283000300DFF1FF0B587B00EAD2F780FAD2D789E
:102840000593AC46634614000E4D0CAA12782E7800
:1028500003930D9B009201932200059B029701F0C8
:102860009BFA2E70012C01D0042C08D1802206493D
:102870008B889343054A1278D20113438B8007B0AB
:10288000F0BDC0461C09FF1F6C11FF1F7809FF1F18
:102890000B001B3B70B504003020E02B0DD813005B
:1028A000E025493BFF3B9BB2ED00AB4205D8034B13
:1028B000200019825A8201F0B7F970BD8410FF1F01
:1028C00010B501F099FA054B00205B68052B04D97F
:1028D000034A5268D20200D4980810BD001000408C
:1028E000FCE100E070B501F0F7F90D4B1B68FC331B
:1028F000DC691D6AFFF7E4FF6419844204D2094BC6
:1029000001241B68002B07D004220024064B1A70F8
:10291000064A93690133936101F056FB200070BDB4
:10292000AC64FF1F9809FF1F2309FF1FFC0FFF1F47
:1029300070B50C4D2B68FC335C6A01F0CDF9FFF7E4
:10294000BFFF2B680025FC339B6AE318834204D247
:10295000054B1B68AB4200D1051B01F035FB28007D
:1029600070BDC046AC64FF1F9809FF1FD722044BFF
:1029700092009B5810B5002B00D0984710BDC04660
:102980000000FF1F10B501F0DBF8FFF7EFFF27494C
:10299000274BCA6D274C1A4084235B001343CB6539
:1029A000254B1B68186A01F067F9244B244A1A600A
:1029B000244B254A1A60A022244B52001A60244B53
:1029C000187801F041FA2000224901F0A5F900230E
:1029D000A3600233A360204B2049236003232048D7
:1029E000A36001F099F910221E4BFF201A6080228B
:1029F00052031A60802292031A60802212041A6025
:102A000001F062FA012001F05FF9FA20400001F0C4
:102A10006BF9582001F028FB134801F0A5FA0120BA
:102A200001F04AF9072001F017FB10BD00F000404B
:102A300000FEFEFF14100040AC64FF1F00000340C6
:102A40000180063DBC00034034080000A4000340A0
:102A50004A0AFF1F71020000C3090000FFFF3F0088
:102A60002810004000E100E030750000674E336838
:102A700088331B6883F3088801F0AEF9644A65491E
:102A8000136800200B401360634B644A1B68934239
:102A900000D1A6E001F090FA0221614A13688B434D
:102AA0001360FFF76FFF5F4B5F4C1878C0B201F007
:102AB000FBF90023A3600233A3605C4B0120236079
:102AC00001F0DAF80323A36001F076F8040001F0C6
:102AD00093F9050001F070F8554B186001F0D4FA35
:102AE000544B1968621A531EA14200D2130080226F
:102AF000D203934201D39B029B0A3268D16AC90771
:102B000000D471E04C491C0C09689BB24C435943FA
:102B10002402090A641803264849FC3293680A68AB
:102B200047489B1A474A0768126847499B18474A13
:102B30009A1833409208DB190A600360042B03D90A
:102B4000013233400A6003600E684149A619300023
:102B500001F032F93F4F3E493B68C3183B603000FB
:102B6000019301F011F93C4E306808183849306083
:102B7000884205D9019B01333B6001F005F93160C2
:102B800001F08AFA354B1B78002B0DD001F034F997
:102B9000334B621B196812188A4232D24919091B39
:102BA000091A304801F0B8F82F4E337A002B0ED0B6
:102BB00001F022F9621BF1681218914224D94919D7
:102BC000091B091A294801F0A7F800233372284B82
:102BD00083F3088801F0C0F9002001F0EDF901F05D
:102BE00003F801F0E9F95CE7DC0199000234641AAA
:102BF0005900641A09214B438033CB40A408E418E0
:102C000089E7FA218900CCE71A49DBE7AC64FF1FAA
:102C10001CF00040FFFFC1FF0C0AFF1FB64121035B
:102C200010000040490AFF1F14100040C3090000B3
:102C3000100AFF1F340AFF1F380AFF1F200AFF1F58
:102C4000280AFF1F1C0AFF1F240AFF1FC4090000D7
:102C5000710200006008FF1F2C0AFF1F1C09FF1FE4
:102C6000E408FF1F00100040740BFF1F3C100040E1
:102C700000000020DC050000A022054B92009B58BC
:102C800010B5002B01D0984710BD01F08DF8FBE77F
:102C90000000FF1FA122054B92009B5810B5002B8E
:102CA00001D0984710BD01F07FF8FBE70000FF1F3F
:102CB000A222054B92009B5810B5002B01D09847DB
:102CC00010BD01F071F8FBE70000FF1FA322054BC8
:102CD00092009B5810B5002B01D0984710BD01F011
:102CE00063F8FBE70000FF1FA422054B92009B58EE
:102CF00010B5002B01D0984710BD01F055F8FBE747
:102D00000000FF1F70B501F077F84F4B186001F01D
:102D100003F90400C30702D401F01EF870BD0022BD
:102D20004A4B1A604A4B18780138042829D800F019
:102D30001FFF0320181C2400200001F0E5F80128E3
:102D4000ECD0444C2378042B6ED100F0FDFF00281A
:102D5000E4D001F021F9582001F086F90223237014
:102D6000DCE7200000F098FFE9E7200001F0BCF864
:102D7000E5E7200000F098FFE1E7200000F0DCFF2D
:102D8000DDE701F011F90500012808D1324B1B786D
:102D9000053B012B03D82000FFF76EFFD1E72D4B39
:102DA0001B78022B01D0052B20D1022D28D12B4BD3
:102DB0009B7BAB431CD12000FFF76CFF264B1878A0
:102DC0000128BED16405BCD4244925224B7B034293
:102DD00005D1233A13405A42534126331A000B7D42
:102DE0009342AED9322000F0FFFFAAE7022D07D1AF
:102DF000194B1B78052B11D12000FFF759FFDDE798
:102E0000012D0BD1012B03D12000FFF75FFF98E7C5
:102E1000062B03D12000FFF767FF92E7200000F0A8
:102E2000C3FF022D8DD1C9E7032B04D10C4B987C35
:102E300001F012F872E7072B00D06FE7094B987B7F
:102E400000F0C2FF6AE7C0469C09FF1F9809FF1FF8
:102E50009009FF1F2309FF1F1C09FF1FA60BFF1F5F
:102E6000BC0BFF1FD40BFF1FFA210A4B0A4A490073
:102E70001A640A4A5A500A4A04395A50094A08310F
:102E80009A64094A5A50094A5C315A50084ADA662B
:102E90007047C0460000FF1F3528FF1F3129FF1F64
:102EA000E528FF1F1524FF1FA527FF1FB51EFF1FC5
:102EB000891EFF1FF7B50B0CFF270122009300238B
:102EC0003C001E001D009446019089B262469A4063
:102ED0001000084018413618B6B2FF2F02D1012E5B
:102EE00000D19FB2009802401A41AD18ADB2FF2C3C
:102EF00002D1012D00D19CB20133102BE6D1032069
:102F0000012E07D1012D04D1019B2401E4191C706D
:102F10000138FEBD102EFCD10238102DF9D0023040
:102F2000F7E700008023F7B59C46264B264F019318
:102F30002649274A274D284C284B02281AD160469B
:102F400038600868264E30408026360330430860DB
:102F500001990978002909D11660224A2A60224A7B
:102F60002260E02219689143A03A1BE08021C90247
:102F70001160F2E766463E600F68194E3E408027BA
:102F8000FF023E430E600199097800290DD11760B8
:102F900001280ED1154A2A60154A2260E0221968DC
:102FA0009143C03A0A431A60F7BD8021890211603B
:102FB000EEE7E0210F4A02432A600F4A22601A68B6
:102FC0008A43F0E74B0AFF1FE0000340D8000340AC
:102FD00090000340000003405000034040000340C5
:102FE000FFFFE3FF0280063D804508220180063D89
:102FF000806608220080069880550822F8B51E4B8E
:1030000080261A68002014003440324232D11A68F7
:103010001A4F32431A6001223B68063093433B60EB
:1030200000F02AFE0122164D2B681E432E603B68DD
:103030000A2613433B608027BF00124B1B683B42AC
:1030400011D1013EF6B2FF2E09D17E220E4B1C6833
:103050002B68E40B1440934323432B6005E00820C6
:1030600000F00AFEE9E7002EEFD180222B6860080D
:1030700093432B60F8BDC046C4F000405CF00040B4
:1030800018F0004068F0004060F0004010B500F01B
:10309000EBFE01215820034A00F0AEFDFFF7AEFF22
:1030A00010BDC046600AFF1F10B5782200210348FA
:1030B00000F002FF00F0D8FD002010BDA067FF1F48
:1030C00070B5040000F008FE00230C200B4A01003C
:1030D00059438D18515C00290DD0A14208D101231C
:1030E00000246B7000F088FF00F06EFF200070BDC0
:1030F00001330A2BEBD11224F6E7C046A067FF1F6D
:1031000070B5040000F0E8FD002319001D000D4A11
:103110001078002806D0A0420CD1557001310C3235
:103120000A29F5D1002B0AD100F09EFD00F04CFFDA
:10313000002070BD5078461EB0411B18EEE700F02D
:103140005BFFF3E7A067FF1FF7B504000C20002327
:1031500084460E4D019267465F43E85D7E19A042AA
:1031600012D000280BD10A4B9C4662461B780833CC
:103170001370019B70707C557160B360FEBD0133AC
:103180000A2BE8D10320F9E70720F7E7A067FF1F24
:103190009C67FF1F8020F8B5484BC0051B68C12401
:1031A0008360474BFF251A68012313434361454B56
:1031B000A4001A68444B40211A60444B1A68444BDF
:1031C0001A60444B1A59AA431A51C52292009E58BC
:1031D000AE433143802699509F583F49F6010F4036
:1031E0003E439E509E5880273602360A3043985000
:1031F00080201A5900020A4002431A5104341A5915
:10320000364E3F04324080263A431A511A59360648
:103210001202120A32431A5108341A5980260A40FF
:1032200002431A51C32292009F58B446AF4337431A
:103230009F509F58294E0F4007439F509F5837403B
:1032400080263604374380269F509F5836063F021B
:103250003F0A37439F50C0221F59AF433A431A5188
:103260001A591202120A1643C6221E5192009C5885
:10327000AC4365462C439C509C5800250C40204391
:103280009850C72080001A58154C1140C0221202D5
:103290000A431A50134B1B78DB08AB4201DC0020B9
:1032A000F8BD2378002B06D0A368002B00D09847E8
:1032B00001350C34EEE71220F2E7C046A043FF1FB1
:1032C0009C43FF1FB0F000409867FF1FB4F0004020
:1032D0009467FF1F00E100E0FF00FFFFFFFF00FF1A
:1032E000A067FF1F9C67FF1F030010B51F2809D8A8
:1032F000072200201340072404490A78A2431343FD
:103300000B7010BD00230620F5E7C0469C67FF1F29
:10331000034A0449136800200B4013607047C046FD
:103320001CF00040FFFFC1FF054B06491B780A68EF
:1033300005485B0702401B0B134300200B607047DE
:103340009C67FF1F1CF00040FFFFC1FF70B50C25FC
:10335000FFF7EAFF0A4B1C780A4BE4086543ED18B7
:10336000002C01D1200070BD2B78002B06D06B689B
:10337000002B00D09847013C0C3DF1E71220F2E70A
:103380009C67FF1F9467FF1F1FB5002102220B00DF
:1033900001910091052000F04FFC02230B490A68BF
:1033A0001A42FCD120230393039B5A1E0392002B45
:1033B000FAD1074A1368002BFCDA0B246C44200076
:1033C000012100F089FD207804B010BD90C80040B4
:1033D00000C8004013B504000A4B0193019B002B69
:1033E00001D1112016BDFFF7CFFF23000340044297
:1033F00005D0052000F040FC019B013BEDE71800E3
:10340000F0E7C046FFFFFF0707B500F065FC80222C
:103410000821D205936A0191002B01D107399162ED
:1034200002210C4A11600199481E01900029FAD12D
:1034300003311160053101910199481E0190002965
:10344000FAD11160002B02D18022D205936200F0E4
:10345000BBFD07BD00C00040F0B52D4C89B02378FE
:10346000002B4FD1FEF7A8FA02232A4F03903A68A7
:103470001A42FCD120230693069B5A1E0692002B6B
:10348000FAD1254E3368002BFCDA0120FFF7A2FFAA
:10349000011E02D0112009B0F0BD030003220190EB
:1034A000009005AD9F2000F0C7FB0321280000F02D
:1034B00013FD02233A681A42FCD120230793079B8D
:1034C0005A1E0792002BFAD13368002BFCDA012038
:1034D000FFF780FF0028DDD10398FEF781FAAA7874
:1034E0006B7811041B020B4329780B4363601300B4
:1034F000113B0A49052B07D801239340A3600B60B9
:10350000012323700020C6E780231B03F6E7C04693
:103510008843FF1F90C8004000C800409808FF1F64
:103520001E4B30B55A6818781D4B85B0D3185942D8
:103530004B4101210093002300F0DEFB194B1A4A96
:1035400002259A6300221A6510325A658022C4212E
:103550009D65164B1648D202DA6789004258154B12
:1035600080241A4080231B041343435064234120CA
:103570000393E40500F006FA402000F003FA6562C8
:10358000039D6B1E0393002DFAD103236362FFF7A3
:103590003BFFA562FFF760FF05B030BD9443FF1FFE
:1035A00095FFFEF700C80040050001FF04E100E0C0
:1035B00000E100E0FFFF00FFF0B585B00700FEF777
:1035C000FBF9022305002D4C22681A42FCD120236E
:1035D0000093009B5A1E0092002BFAD1284E3368AC
:1035E000002BFCDA0120FFF7F5FE002803D01124A0
:1035F000200005B0F0BD234B2360022322681A424D
:10360000FCD120230193019B5A1E0192002BFAD179
:103610003368002BFCDA0120FFF7DCFE0028E6D13E
:10362000194B1F60022322681A42FCD12023029307
:10363000029B5A1E0292002BFAD13368002BFCDA4F
:103640000120FFF7C7FE0028D1D1104B23600223D1
:1036500022681A42FCD120230393039B5A1E039233
:10366000002BFAD13368002BFCDA0120FFF7B2FE01
:10367000041EBCD12800FEF7B3F9B9E790C800409A
:1036800000C8004001000006A8C8004001800001F9
:1036900010B50020FFF790FF10BD000010B5064BDD
:1036A00018705960FFF73CFF00211320034AFFF711
:1036B0004BFD002010BDC0469443FF1F2135FF1F66
:1036C000F0B5040085B003920291FEF775F98822E7
:1036D00063035B0B52051A438023DB059D6A80233D
:1036E000274F0092BA68002601901B039A420CD91A
:1036F000F82326001B041E401C4206D08022214BCA
:1037000052025E6219680A431A60002D0BD100F064
:10371000E3FA02221C4B1A608023DB055A62013A4D
:103720009A6200F051FC0023039A934220D1002DAD
:103730000AD100F0D1FA144B03221D608023DB056F
:103740005A629D6200F040FC8023BA681B039A42D3
:1037500008D9002E06D000220A4B0C495A621A687A
:103760000A401A600198FEF73BF9002005B0F0BD51
:10377000009A0299D2181278CA540133D4E7C0468D
:103780008843FF1F00C8004000C00040FFFFFEFF4D
:10379000F0B587B0029103920400FEF70DF9019095
:1037A00000F09AFA802302250122234EDB053560C2
:1037B0005D629A6200F008FC204F3B682B42FCD10E
:1037C00020230493049B5A1E0492002BFAD11C4D13
:1037D0002B68002BFCDA0120FFF7FCFD002802D04B
:1037E000112007B0F0BD2000039A029900F0C4FB3D
:1037F000022304003A681A42FCD120230593059B5A
:103800005A1E0592002BFAD12B68002BFCDA0120FE
:10381000FFF7E0FD051EE3D100F05EFA80230322EE
:10382000DB0535605A629D6200F0CEFB0198FEF721
:10383000D7F8E0B2D5E7C04600C0004090C80040CD
:1038400000C80040F0B5802489B00600FEF7B4F847
:10385000E405A36A02250393029000F03DFA0123D8
:10386000304F3D606562A36200F0AEFB2E4C2368D2
:103870002B42FCD120230593059B5A1E0592002B59
:10388000FAD12A4D2B68002BFCDA0120FFF7A2FDAC
:10389000002803D01124200009B0F0BD244B236080
:1038A000022322681A42FCD120230693069B5A1E4B
:1038B0000692002BFAD12B68002BFCDA0120FFF7CF
:1038C00089FD021EE6D11B4B03211E6003000190FF
:1038D0000090202000F0B0F9022322681A42FCD1A7
:1038E00020230793079B5A1E0792002BFAD12B68BF
:1038F000002BFCDA0320FFF76DFD041ECAD100F097
:10390000EBF980230322DB053C605A629C6200F0E5
:103910005BFB039B002B01D1FFF776FD0298FEF7BE
:103920005FF8B8E700C0004090C8004000C8004001
:103930000100000694C8004007B50002019104226E
:10394000000A01A9FFF724FF0EBD000073B50500B2
:1039500005240B4AA3005B429B1819686B46DE1DC9
:103960003000FFF7A7FA022804D133782B55013C29
:10397000EFD276BD052CFCD00128FAD10230F8E751
:10398000140900111F2807D8012380228340D20583
:1039900091680B43936070473F2808D80123802229
:1039A00020388340D20551690B435361F3E75F2808
:1039B000F1D80123802240388340D205116A0B439D
:1039C0001362E8E71F2807D8012280218240C90539
:1039D0008B6893438B6070473F2808D80122802171
:1039E00020388240C9054B6993434B61F3E75F2858
:1039F000F1D80122802140388240C9050B6A9343E7
:103A00000B62E8E71F2810D880230200DB05153A77
:103A10001968012A06D820229143196019680A43BF
:103A20001A60704701228240F6E73F2811D88023B0
:103A30000200DB05353AD968032A06D810229143E3
:103A4000D960D9680A43DA60EBE701222038824066
:103A5000F5E75F28E5D842238022181A413B8340CE
:103A6000D205516A99435162516A0B435362D8E7B8
:103A700010B50400012813D1A022184992050B6843
:103A80005B015B0913430B60154B164A1968114023
:103A9000154A0A431A60402219680A431A6010BD89
:103AA0000028FCD101000A2000F06EFA21000B2052
:103AB00000F06AFAC0220A4B920019680A434021BA
:103AC0001A601A688A431A60B022044912060B6809
:103AD0005B015B0913430B60E1E7C04614F0004053
:103AE0001CF000407F00FEFF80FD010072B6074A17
:103AF0001368013313600422054B1A600023054A42
:103B000013608022D2055360FEE7C0467808FF1F8D
:103B1000C0F00040C4F0004005490B68002B05D1FF
:103B2000044A0A6004490A60044A13607047C046A8
:103B3000140AFF1F841E0000380AFF1FC4F0004053
:103B40000023034A1360034A1360034A136070475B
:103B500054F0004040F1004044F1004002B471468E
:103B600049084900095649008E4402BC7047C046C6
:103B700002B4714649084900095C49008E4402BC00
:103B80007047C04603B47146490840004900095ACD
:103B900049008E4403BC704701B40248844601BC0E
:103BA000604700BF5976010001B40248844601BC59
:103BB000604700BF75F8000001B40248844601BCAC
:103BC000604700BF156B010001B40248844601BC88
:103BD000604700BF8944000001B40248844601BC2C
:103BE000604700BFE927000001B40248844601BCD9
:103BF000604700BF8552010001B40248844601BC01
:103C0000604700BF0167010001B40248844601BC5F
:103C1000604700BFA1AF000001B40248844601BC68
:103C2000604700BFF9ED000001B40248844601BCC2
:103C3000604700BF116E000001B40248844601BC19
:103C4000604700BF496D010001B40248844601BCD1
:103C5000604700BFC1A5000001B40248844601BC12
:103C6000604700BF0D52010001B40248844601BC08
:103C7000604700BFADAE000001B40248844601BCFD
:103C8000604700BF0189000001B40248844601BCBE
:103C9000604700BF51B8000001B40248844601BC2F
:103CA000604700BF0934010001B40248844601BCEA
:103CB000604700BFF535010001B40248844601BCED
:103CC000604700BFE512010001B40248844601BC10
:103CD000604700BF6911010001B40248844601BC7D
:103CE000604700BF75A9000001B40248844601BCCA
:103CF000604700BF8512010001B40248844601BC40
:103D0000604700BFC56D010001B40248844601BC94
:103D1000604700BF6D0B010001B40248844601BC3E
:103D2000604700BF2D6C010001B40248844601BC0D
:103D3000604700BFE9D4000001B40248844601BCDA
:103D4000604700BFF935010001B40248844601BC58
:103D5000604700BF01D7000001B40248844601BC9F
:103D6000604700BFDD0A010001B40248844601BC7F
:103D7000604700BFBD5C010001B40248844601BC3D
:103D8000604700BF85C1000001B40248844601BC01
:103D9000604700BF090E000001B40248844601BC20
:103DA000604700BF9D6A000001B40248844601BC20
:103DB000604700BFE917010001B40248844601BC16
:103DC000604700BF090E000001B40248844601BCF0
:103DD000604700BFC1F7000001B40248844601BC3F
:103DE000604700BFC9A9000001B40248844601BC75
:103DF000604700BF6137010001B40248844601BC3E
:103E0000604700BFC95C010001B40248844601BCA0
:103E1000604700BFE9F6000001B40248844601BCD7
:103E2000604700BFCD0C010001B40248844601BCCC
:103E3000604700BF8B52010001B40248844601BCB8
:103E4000604700BF8937010001B40248844601BCC5
:103E5000604700BFEDA5000001B40248844601BCE4
:103E6000604700BF4DF9000001B40248844601BC20
:103E7000604700BFED68010001B40248844601BC00
:103E8000604700BFE90B010001B40248844601BC51
:103E9000604700BFDD3F000001B40248844601BC1A
:103EA000604700BFD1AE000001B40248844601BCA7
:103EB000604700BF8914010001B40248844601BC78
:103EC000604700BFB70E000001B40248844601BC41
:103ED000604700BFED6B010001B40248844601BC9D
:103EE000604700BF3D71010001B40248844601BC37
:103EF000604700BF0534010001B40248844601BC9C
:103F0000604700BFCD4C010001B40248844601BCAB
:103F1000604700BF0134010001B40248844601BC7F
:103F2000604700BFBD0B010001B40248844601BCDC
:103F3000604700BF71B0000001B40248844601BC74
:103F4000604700BFE94C010001B40248844601BC4F
:103F5000604700BF8D82000001B40248844601BC66
:103F6000604700BF7997000001B40248844601BC55
:103F7000604700BF8D11010001B40248844601BCB6
:103F8000604700BF9573010001B40248844601BC3C
:103F9000604700BFB5A3001101B40248844601BCCC
:103FA000604700BF6DF6000001B40248844601BCC2
:103FB000604700BFDD0C010001B40248844601BC2B
:103FC000604700BF016C010001B40248844601BC97
:103FD000604700BF9DA9000001B40248844601BCAF
:103FE000604700BFB352010001B40248844601BCDF
:103FF000604700BF53B9000001B40248844601BCC9
:10400000604700BF21A9000001B40248844601BCFA
:10401000604700BFC115010001B40248844601BCDD
:10402000604700BFD9B0000001B40248844601BC1B
:10403000604700BF5DB7001101B40248844601BC6F
:10404000604700BFA9D8000001B40248844601BC03
:10405000604700BF19FA000001B40248844601BC61
:10406000604700BFF90D010001B40248844601BC5D
:10407000604700BF7912010001B40248844601BCC8
:10408000604700BF2144000001B40248844601BCDF
:10409000604700BFC166010001B40248844601BC0C
:0840A000604700BFD544010098
:1040A800020000002AC000110100000020BE00111B
:1040B8000200000026C0001101000000E840FF1FB8
:1040C8000200000028BE0011010000001C62FF1F52
:1040D8000200000024C00011030000009061FF1FCF
:1040E80012000000020000002AC0001101000000B8
:1040F80068BE00110200000026C000110100000087
:1041080065BE00110200000072BE0011030000002D
:10411800CB61FF1F0200000024C000110300000053
:10412800E061FF1F0200000026C00011010000002E
:1041380064BE00110200000070BE00110300000000
:10414800A161FF1F0200000024C00011030000004D
:10415800C261FF1F020000002AC000110100000018
:10416800A8BE00110200000026C0001101000000D6
:104178003142FF1F02000000BABE0011010000001A
:10418800A3BE00110200000026C0001101000000BB
:104198003042FF1F02000000B8BE001101000000FD
:1041A800E861FF1F0200000026C0001101000000A6
:1041B8002F42FF1F02000000B6BE001101000000E0
:1041C80093BE00110200000026C00011010000008B
:1041D8002E42FF1F02000000B4BE001101000000C3
:1041E8008EBE00110200000026C000110100000070
:1041F8002D42FF1F02000000B2BE001101000000A6
:1042080089BE00110200000026C000110100000054
:104218002C42FF1F02000000B0BE00110100000088
:1042280084BE001102020202020200000000000027
:1042380016150000E14C0011A74C001118BF001121
:1042480090011D0018001800FFFF07010203040574
:104258000602010600000000000000000000000047
:104268000000000000000000000000000000000046
:1042780003000000020000002AC000110100000035
:1042880038BF00110200000026C000110100000024
:10429800EC42FF1F0200000042BF001101000000B5
:1042A8001662FF1F0200000024C000110300000076
:1042B8008064FF1F0200000026C0001101000000FA
:1042C800EC42FF1F0200000040BF00110100000087
:1042D8001862FF1F0200000024C000110300000044
:1042E8007864FF1F1200000000000000161500008F
:1042F8000001000000000111FFFF0000504859367E
:1043080000000000000000000B000500F0000000A5
:10431800B4000028002800283075A000A000A000E4
:10432800A00000080008E001F000100010001000D4
:104338001000100010005000500050001000100035
:10434800D0070000000000000F00010005003075D4
:1043580007001000010081FF00000000FF000000BE
:104368009D750011A573001135710011FFFF010043
:10437800FF000000B99F0011359D00114D9C0011F0
:104388000000000000000000000008000400000019
:104398003B0001085902E00188212800FF000000C5
:1043A800020000002AC0001101000000F0C0001146
:1043B8000200000026C00011010000002544FF1F74
:1043C8000200000022C00011010000005868FF1F11
:1043D8000200000026C00011010000002444FF1F55
:1043E8000200000020C00011010000002244FF1F4D
:1043F8000200000026C00011010000002044FF1F39
:10440800020000001EC00011010000001844FF1F38
:10441800180018001D0090010200000302020000AD
:10442800020000002AC000110100000004C10011B0
:104438000200000026C00011010000006844FF1FB0
:10444800020000001CC00011000000000000000075
:104458000200000024C00011030000007868FF1F5C
:0244680020FF33
:040000051FFF184180
:00000001FF
